 jaccessinspector

 Timestamp is ffffffff (Sun Feb  7 06:28:15 2106)

 Preferred load address is 00400000

 Start         Length     Name                   Class
 0001:00000000 00000020H .text$di                CODE
 0001:00000020 0000c610H .text$mn                CODE
 0001:0000c630 00000120H .text$x                 CODE
 0001:0000c750 0000000fH .text$yd                CODE
 0002:00000000 0000022cH .idata$5                DATA
 0002:0000022c 00000004H .00cfg                  DATA
 0002:00000230 00000004H .CRT$XCA                DATA
 0002:00000234 00000004H .CRT$XCAA               DATA
 0002:00000238 00000004H .CRT$XCU                DATA
 0002:0000023c 00000004H .CRT$XCZ                DATA
 0002:00000240 00000004H .CRT$XIA                DATA
 0002:00000244 00000004H .CRT$XIAA               DATA
 0002:00000248 00000004H .CRT$XIAC               DATA
 0002:0000024c 00000004H .CRT$XIC                DATA
 0002:00000250 00000004H .CRT$XIZ                DATA
 0002:00000254 00000004H .CRT$XLA                DATA
 0002:00000258 00000004H .CRT$XLZ                DATA
 0002:0000025c 00000004H .CRT$XPA                DATA
 0002:00000260 00000004H .CRT$XPZ                DATA
 0002:00000264 00000004H .CRT$XTA                DATA
 0002:00000268 00000008H .CRT$XTZ                DATA
 0002:0000026c 00000000H .gfids$y                DATA
 0002:00000270 00002108H .rdata                  DATA
 0002:00002378 00000018H .rdata$T                DATA
 0002:00002390 0000012cH .rdata$r                DATA
 0002:000024bc 00000020H .rdata$sxdata           DATA
 0002:000024dc 000003b0H .rdata$zzzdbg           DATA
 0002:0000288c 00000004H .rtc$IAA                DATA
 0002:00002890 00000004H .rtc$IZZ                DATA
 0002:00002894 00000004H .rtc$TAA                DATA
 0002:00002898 00000004H .rtc$TZZ                DATA
 0002:0000289c 00000004H .tls                    DATA
 0002:000028a0 00000004H .tls$                   DATA
 0002:000028a4 00000004H .tls$ZZZ                DATA
 0002:000028a8 00000178H .xdata$x                DATA
 0002:00002a20 00000000H .edata                  DATA
 0002:00002a20 00000104H .idata$2                DATA
 0002:00002b24 00000014H .idata$3                DATA
 0002:00002b38 0000022cH .idata$4                DATA
 0002:00002d64 00000a40H .idata$6                DATA
 0003:00000000 00000aa8H .data                   DATA
 0003:00000aa8 00000078H .data$r                 DATA
 0003:00000b20 00000750H .bss                    DATA
 0004:00000000 000001c0H .rsrc$01                DATA
 0004:000001c0 00000ec8H .rsrc$02                DATA

  Address         Publics by Value              Rva+Base       Lib:Object

 0000:00000000       ___guard_longjmp_table     00000000     <absolute>
 0000:00000000       ___hybrid_code_map_count   00000000     <absolute>
 0000:00000000       ___guard_iat_table         00000000     <absolute>
 0000:00000000       ___guard_eh_cont_count     00000000     <absolute>
 0000:00000000       ___arm64x_redirection_metadata 00000000     <absolute>
 0000:00000000       ___arm64x_extra_rfe_table_size 00000000     <absolute>
 0000:00000000       ___hybrid_auxiliary_iat    00000000     <absolute>
 0000:00000000       ___hybrid_code_map         00000000     <absolute>
 0000:00000000       ___volatile_metadata       00000000     <absolute>
 0000:00000000       ___AbsoluteZero            00000000     <absolute>
 0000:00000000       ___enclave_config          00000000     <absolute>
 0000:00000000       ___arm64x_extra_rfe_table  00000000     <absolute>
 0000:00000000       ___guard_eh_cont_table     00000000     <absolute>
 0000:00000000       ___arm64x_redirection_metadata_count 00000000     <absolute>
 0000:00000000       ___guard_iat_count         00000000     <absolute>
 0000:00000000       ___x64_code_ranges_to_entry_points_count 00000000     <absolute>
 0000:00000000       ___guard_fids_table        00000000     <absolute>
 0000:00000000       ___dynamic_value_reloc_table 00000000     <absolute>
 0000:00000000       ___guard_longjmp_count     00000000     <absolute>
 0000:00000000       ___guard_fids_count        00000000     <absolute>
 0000:00000000       ___arm64x_native_entrypoint 00000000     <absolute>
 0000:00000000       ___x64_code_ranges_to_entry_points 00000000     <absolute>
 0000:00000008       ___safe_se_handler_count   00000008     <absolute>
 0000:0000002c       __tls_array                0000002c     <absolute>
 0000:00000100       ___guard_flags             00000100     <absolute>
 0000:00000000       ___ImageBase               00400000     <linker-defined>
 0001:00000020       _initializeAccessBridge    00401020 f   AccessBridgeCalls.obj
 0001:00000ee0       _shutdownAccessBridge      00401ee0 f   AccessBridgeCalls.obj
 0001:00000f30       _IsJavaWindow              00401f30 f   AccessBridgeCalls.obj
 0001:00000f60       _GetAccessibleContextFromHWND 00401f60 f   AccessBridgeCalls.obj
 0001:00000f90       _getHWNDFromAccessibleContext 00401f90 f   AccessBridgeCalls.obj
 0001:00000fc0       _SetJavaShutdown           00401fc0 f   AccessBridgeCalls.obj
 0001:00000fe0       _SetFocusGained            00401fe0 f   AccessBridgeCalls.obj
 0001:00001000       _SetFocusLost              00402000 f   AccessBridgeCalls.obj
 0001:00001020       _SetCaretUpdate            00402020 f   AccessBridgeCalls.obj
 0001:00001040       _SetMouseClicked           00402040 f   AccessBridgeCalls.obj
 0001:00001060       _SetMouseEntered           00402060 f   AccessBridgeCalls.obj
 0001:00001080       _SetMouseExited            00402080 f   AccessBridgeCalls.obj
 0001:000010a0       _SetMousePressed           004020a0 f   AccessBridgeCalls.obj
 0001:000010c0       _SetMouseReleased          004020c0 f   AccessBridgeCalls.obj
 0001:000010e0       _SetMenuCanceled           004020e0 f   AccessBridgeCalls.obj
 0001:00001100       _SetMenuDeselected         00402100 f   AccessBridgeCalls.obj
 0001:00001120       _SetMenuSelected           00402120 f   AccessBridgeCalls.obj
 0001:00001140       _SetPopupMenuCanceled      00402140 f   AccessBridgeCalls.obj
 0001:00001160       _SetPopupMenuWillBecomeInvisible 00402160 f   AccessBridgeCalls.obj
 0001:00001180       _SetPopupMenuWillBecomeVisible 00402180 f   AccessBridgeCalls.obj
 0001:000011a0       _SetPropertyNameChange     004021a0 f   AccessBridgeCalls.obj
 0001:000011c0       _SetPropertyDescriptionChange 004021c0 f   AccessBridgeCalls.obj
 0001:000011e0       _SetPropertyStateChange    004021e0 f   AccessBridgeCalls.obj
 0001:00001200       _SetPropertyValueChange    00402200 f   AccessBridgeCalls.obj
 0001:00001220       _SetPropertySelectionChange 00402220 f   AccessBridgeCalls.obj
 0001:00001240       _SetPropertyTextChange     00402240 f   AccessBridgeCalls.obj
 0001:00001260       _SetPropertyCaretChange    00402260 f   AccessBridgeCalls.obj
 0001:00001280       _SetPropertyVisibleDataChange 00402280 f   AccessBridgeCalls.obj
 0001:000012a0       _SetPropertyChildChange    004022a0 f   AccessBridgeCalls.obj
 0001:000012c0       _SetPropertyActiveDescendentChange 004022c0 f   AccessBridgeCalls.obj
 0001:000012e0       _SetPropertyTableModelChange 004022e0 f   AccessBridgeCalls.obj
 0001:00001300       _ReleaseJavaObject         00402300 f   AccessBridgeCalls.obj
 0001:00001320       _GetVersionInfo            00402320 f   AccessBridgeCalls.obj
 0001:00001350       _GetAccessibleContextAt    00402350 f   AccessBridgeCalls.obj
 0001:00001380       _GetAccessibleContextWithFocus 00402380 f   AccessBridgeCalls.obj
 0001:000013b0       _GetAccessibleContextInfo  004023b0 f   AccessBridgeCalls.obj
 0001:000013e0       _GetAccessibleChildFromContext 004023e0 f   AccessBridgeCalls.obj
 0001:00001410       _GetAccessibleParentFromContext 00402410 f   AccessBridgeCalls.obj
 0001:00001440       _GetAccessibleTextInfo     00402440 f   AccessBridgeCalls.obj
 0001:00001470       _GetAccessibleTextItems    00402470 f   AccessBridgeCalls.obj
 0001:000014a0       _GetAccessibleTextSelectionInfo 004024a0 f   AccessBridgeCalls.obj
 0001:000014d0       _GetAccessibleTextAttributes 004024d0 f   AccessBridgeCalls.obj
 0001:00001500       _GetAccessibleTextRect     00402500 f   AccessBridgeCalls.obj
 0001:00001530       _GetAccessibleTextLineBounds 00402530 f   AccessBridgeCalls.obj
 0001:00001560       _GetAccessibleTextRange    00402560 f   AccessBridgeCalls.obj
 0001:000015a0       _getAccessibleTableInfo    004025a0 f   AccessBridgeCalls.obj
 0001:000015d0       _getAccessibleTableCellInfo 004025d0 f   AccessBridgeCalls.obj
 0001:00001600       _getAccessibleTableRowHeader 00402600 f   AccessBridgeCalls.obj
 0001:00001630       _getAccessibleTableColumnHeader 00402630 f   AccessBridgeCalls.obj
 0001:00001660       _getAccessibleTableRowDescription 00402660 f   AccessBridgeCalls.obj
 0001:00001690       _getAccessibleTableColumnDescription 00402690 f   AccessBridgeCalls.obj
 0001:000016c0       _getAccessibleTableRowSelectionCount 004026c0 f   AccessBridgeCalls.obj
 0001:000016f0       _isAccessibleTableRowSelected 004026f0 f   AccessBridgeCalls.obj
 0001:00001720       _getAccessibleTableRowSelections 00402720 f   AccessBridgeCalls.obj
 0001:00001750       _getAccessibleTableColumnSelectionCount 00402750 f   AccessBridgeCalls.obj
 0001:00001780       _isAccessibleTableColumnSelected 00402780 f   AccessBridgeCalls.obj
 0001:000017b0       _getAccessibleTableColumnSelections 004027b0 f   AccessBridgeCalls.obj
 0001:000017e0       _getAccessibleTableRow     004027e0 f   AccessBridgeCalls.obj
 0001:00001810       _getAccessibleTableColumn  00402810 f   AccessBridgeCalls.obj
 0001:00001840       _getAccessibleTableIndex   00402840 f   AccessBridgeCalls.obj
 0001:00001870       _getAccessibleRelationSet  00402870 f   AccessBridgeCalls.obj
 0001:000018a0       _getAccessibleHypertext    004028a0 f   AccessBridgeCalls.obj
 0001:000018d0       _activateAccessibleHyperlink 004028d0 f   AccessBridgeCalls.obj
 0001:00001900       _getAccessibleHyperlinkCount 00402900 f   AccessBridgeCalls.obj
 0001:00001930       _getAccessibleHypertextExt 00402930 f   AccessBridgeCalls.obj
 0001:00001960       _getAccessibleHypertextLinkIndex 00402960 f   AccessBridgeCalls.obj
 0001:00001990       _getAccessibleHyperlink    00402990 f   AccessBridgeCalls.obj
 0001:000019c0       _getAccessibleKeyBindings  004029c0 f   AccessBridgeCalls.obj
 0001:000019f0       _getAccessibleIcons        004029f0 f   AccessBridgeCalls.obj
 0001:00001a20       _getAccessibleActions      00402a20 f   AccessBridgeCalls.obj
 0001:00001a50       _doAccessibleActions       00402a50 f   AccessBridgeCalls.obj
 0001:00001a80       _IsSameObject              00402a80 f   AccessBridgeCalls.obj
 0001:00001ab0       _setTextContents           00402ab0 f   AccessBridgeCalls.obj
 0001:00001ae0       _getParentWithRole         00402ae0 f   AccessBridgeCalls.obj
 0001:00001b10       _getParentWithRoleElseRoot 00402b10 f   AccessBridgeCalls.obj
 0001:00001b40       _getTopLevelObject         00402b40 f   AccessBridgeCalls.obj
 0001:00001b70       _getObjectDepth            00402b70 f   AccessBridgeCalls.obj
 0001:00001ba0       _getActiveDescendent       00402ba0 f   AccessBridgeCalls.obj
 0001:00001bd0       _GetCurrentAccessibleValueFromContext 00402bd0 f   AccessBridgeCalls.obj
 0001:00001c00       _GetMaximumAccessibleValueFromContext 00402c00 f   AccessBridgeCalls.obj
 0001:00001c30       _GetMinimumAccessibleValueFromContext 00402c30 f   AccessBridgeCalls.obj
 0001:00001c60       _GetAccessibleSelectionFromContext 00402c60 f   AccessBridgeCalls.obj
 0001:00001c90       _GetAccessibleSelectionCountFromContext 00402c90 f   AccessBridgeCalls.obj
 0001:00001cc0       _IsAccessibleChildSelectedFromContext 00402cc0 f   AccessBridgeCalls.obj
 0001:00001cf0       _RemoveAccessibleSelectionFromContext 00402cf0 f   AccessBridgeCalls.obj
 0001:00001d20       _SelectAllAccessibleSelectionFromContext 00402d20 f   AccessBridgeCalls.obj
 0001:00001d40       _getVirtualAccessibleName  00402d40 f   AccessBridgeCalls.obj
 0001:00001d70       _requestFocus              00402d70 f   AccessBridgeCalls.obj
 0001:00001da0       _selectTextRange           00402da0 f   AccessBridgeCalls.obj
 0001:00001dd0       _getTextAttributesInRange  00402dd0 f   AccessBridgeCalls.obj
 0001:00001e10       _getVisibleChildrenCount   00402e10 f   AccessBridgeCalls.obj
 0001:00001e40       _getVisibleChildren        00402e40 f   AccessBridgeCalls.obj
 0001:00001e70       _setCaretPosition          00402e70 f   AccessBridgeCalls.obj
 0001:00001ea0       _getCaretLocation          00402ea0 f   AccessBridgeCalls.obj
 0001:00001ed0       _getEventsWaiting          00402ed0 f   AccessBridgeCalls.obj
 0001:00001ef0       _addAccessibleSelectionFromContext 00402ef0 f   AccessBridgeCalls.obj
 0001:00001f20       _clearAccessibleSelectionFromContext 00402f20 f   AccessBridgeCalls.obj
 0001:00001f50       _printError                00402f50 f   AccessBridgeDebug.obj
 0001:00002060       _PrintDebugString          00403060 f   AccessBridgeDebug.obj
 0001:000020d0       _wPrintJavaDebugString     004030d0 f   AccessBridgeDebug.obj
 0001:00002140       _wPrintDebugString         00403140 f   AccessBridgeDebug.obj
 0001:000021b0       _initializeFileLogger      004031b0 f   AccessBridgeDebug.obj
 0001:000022e0       _finalizeFileLogger        004032e0 f   AccessBridgeDebug.obj
 0001:00002310       _getTimeStamp              00403310 f   AccessBridgeDebug.obj
 0001:00002350       _PrintJavaDebugString2     00403350 f   AccessBridgeDebug.obj
 0001:000023c0       ___local_stdio_printf_options 004033c0 f i AccessBridgeDebug.obj
 0001:000023d0       __vfprintf_l               004033d0 f i AccessBridgeDebug.obj
 0001:00002400       __vfwprintf_l              00403400 f i AccessBridgeDebug.obj
 0001:00002430       _fprintf                   00403430 f i AccessBridgeDebug.obj
 0001:00002470       _printf                    00403470 f i AccessBridgeDebug.obj
 0001:000024b0       _vfprintf                  004034b0 f i AccessBridgeDebug.obj
 0001:000024d0       _vfwprintf                 004034d0 f i AccessBridgeDebug.obj
 0001:000024f0       ?initBroadcastMessageIDs@@YAHXZ 004034f0 f   AccessBridgeMessages.obj
 0001:00002540       ?getTimeAndDate@@YAPADXZ   00403540 f   AccessInfo.obj
 0001:000025f0       ?displayAndLog@@YAXPAUHWND__@@HPAU_iobuf@@PADZZ 004035f0 f   AccessInfo.obj
 0001:000026d0       ?logString@@YAXPAU_iobuf@@PADZZ 004036d0 f   AccessInfo.obj
 0001:00002760       ?getAccessibleInfo@@YAPADJPAV_jobject@@PADH@Z 00403760 f   AccessInfo.obj
 0001:00002790       ?getAccessibleInfo@@YAPADJPAV_jobject@@HHPADH@Z 00403790 f   AccessInfo.obj
 0001:00004820       ?appendToBuffer@@YAHPADI0ZZ 00405820 f   AccessInfo.obj
 0001:00004900       __vsnprintf_l              00405900 f i AccessInfo.obj
 0001:00004960       __vsprintf_l               00405960 f i AccessInfo.obj
 0001:00004980       _sprintf                   00405980 f i AccessInfo.obj
 0001:000049c0       _vsprintf                  004059c0 f i AccessInfo.obj
 0001:000049e0       ?AddMessage@MessageHistory@@QAEXPBD@Z 004059e0 f   MessageHistory.obj
 0001:00004ab0       ?GetFirstMessage@MessageHistory@@QAEPBDXZ 00405ab0 f   MessageHistory.obj
 0001:00004b00       ?GetPreviousMessage@MessageHistory@@QAEPBDXZ 00405b00 f   MessageHistory.obj
 0001:00004b60       ?GetNextMessage@MessageHistory@@QAEPBDXZ 00405b60 f   MessageHistory.obj
 0001:00004bd0       ?GetLastMessage@MessageHistory@@QAEPBDXZ 00405bd0 f   MessageHistory.obj
 0001:00004c30       ?GetCurrentMessage@MessageHistory@@QAEPBDXZ 00405c30 f   MessageHistory.obj
 0001:00004c70       ?GetMessageA@MessageHistory@@QAEPBDI@Z 00405c70 f   MessageHistory.obj
 0001:00004cf0       ?GetCurrentMessageIndex@MessageHistory@@QAEIXZ 00405cf0 f   MessageHistory.obj
 0001:00004d40       ?IsFirstMessage@MessageHistory@@QAEHXZ 00405d40 f   MessageHistory.obj
 0001:00004d90       ?IsLastMessage@MessageHistory@@QAEHXZ 00405d90 f   MessageHistory.obj
 0001:00004df0       ?GetMessageCount@MessageHistory@@QAEIXZ 00405df0 f   MessageHistory.obj
 0001:00004e10       ?clear@MessageHistory@@QAEXXZ 00405e10 f   MessageHistory.obj
 0001:00004e30       ??$?0$$V@?$_Compressed_pair@V?$allocator@D@std@@V?$_String_val@U?$_Simple_types@D@std@@@2@$00@std@@QAE@U_Zero_then_variadic_args_t@1@@Z 00405e30 f i MessageHistory.obj
 0001:00004e50       ??$?0V?$allocator@D@std@@$$V@?$_Compressed_pair@V?$allocator@D@std@@V?$_String_val@U?$_Simple_types@D@std@@@2@$00@std@@QAE@U_One_then_variadic_args_t@1@$$QAV?$allocator@D@1@@Z 00405e50 f i MessageHistory.obj
 0001:00004e80       ??$?0V?$basic_string@DU?$char_traits@D@std@@V?$allocator@D@2@@std@@@?$_List_node_emplace_op2@V?$allocator@U?$_List_node@V?$basic_string@DU?$char_traits@D@std@@V?$allocator@D@2@@std@@PAX@std@@@std@@@std@@QAE@AAV?$allocator@U?$_List_node@V?$basic_string@DU?$char_traits@D@std@@V?$allocator@D@2@@std@@PAX@std@@@1@$$QAV?$basic_string@DU?$char_traits@D@std@@V?$allocator@D@2@@1@@Z 00405e80 f i MessageHistory.obj
 0001:00004f10       ??$_Destroy_in_place@PAD@std@@YAXAAPAD@Z 00405f10 f i MessageHistory.obj
 0001:00004f10       ??$_Destroy_in_place@PAU?$_List_node@V?$basic_string@DU?$char_traits@D@std@@V?$allocator@D@2@@std@@PAX@std@@@std@@YAXAAPAU?$_List_node@V?$basic_string@DU?$char_traits@D@std@@V?$allocator@D@2@@std@@PAX@0@@Z 00405f10 f i MessageHistory.obj
 0001:00004f10       ??$_Adl_verify_range@V?$_List_const_iterator@V?$_List_val@U?$_List_simple_types@V?$basic_string@DU?$char_traits@D@std@@V?$allocator@D@2@@std@@@std@@@std@@@std@@V12@@std@@YAXABV?$_List_const_iterator@V?$_List_val@U?$_List_simple_types@V?$basic_string@DU?$char_traits@D@std@@V?$allocator@D@2@@std@@@std@@@std@@@0@0@Z 00405f10 f i MessageHistory.obj
 0001:00004f20       ??$_Allocate@$07U_Default_allocate_traits@std@@$0A@@std@@YAPAXI@Z 00405f20 f i MessageHistory.obj
 0001:00004f60       ??$_Allocate_manually_vector_aligned@U_Default_allocate_traits@std@@@std@@YAPAXI@Z 00405f60 f i MessageHistory.obj
 0001:00004fd0       ??$_Construct_in_place@PAU?$_List_node@V?$basic_string@DU?$char_traits@D@std@@V?$allocator@D@2@@std@@PAX@std@@AAPAU12@@std@@YAXAAPAU?$_List_node@V?$basic_string@DU?$char_traits@D@std@@V?$allocator@D@2@@std@@PAX@0@0@Z 00405fd0 f i jaccessinspector.obj
 0001:00004fd0       ??$_Construct_in_place@PADABQAD@std@@YAXAAPADABQAD@Z 00405fd0 f i MessageHistory.obj
 0001:00004fd0       ??$_Construct_in_place@PAU?$_List_node@V?$basic_string@DU?$char_traits@D@std@@V?$allocator@D@2@@std@@PAX@std@@ABQAU12@@std@@YAXAAPAU?$_List_node@V?$basic_string@DU?$char_traits@D@std@@V?$allocator@D@2@@std@@PAX@0@ABQAU10@@Z 00405fd0 f i MessageHistory.obj
 0001:00005010       ??$_Convert_size@I@std@@YAII@Z 00406010 f i MessageHistory.obj
 0001:00005010       ??$forward@AAPAU?$_List_node@V?$basic_string@DU?$char_traits@D@std@@V?$allocator@D@2@@std@@PAX@std@@@std@@YAAAPAU?$_List_node@V?$basic_string@DU?$char_traits@D@std@@V?$allocator@D@2@@std@@PAX@0@AAPAU10@@Z 00406010 f i jaccessinspector.obj
 0001:00005010       ??$forward@ABQAU?$_List_node@V?$basic_string@DU?$char_traits@D@std@@V?$allocator@D@2@@std@@PAX@std@@@std@@YAABQAU?$_List_node@V?$basic_string@DU?$char_traits@D@std@@V?$allocator@D@2@@std@@PAX@0@ABQAU10@@Z 00406010 f i MessageHistory.obj
 0001:00005010       ??$addressof@PAD@std@@YAPAPADAAPAD@Z 00406010 f i MessageHistory.obj
 0001:00005010       ??$move@AAV?$_List_const_iterator@V?$_List_val@U?$_List_simple_types@V?$basic_string@DU?$char_traits@D@std@@V?$allocator@D@2@@std@@@std@@@std@@@std@@@std@@YA$$QAV?$_List_const_iterator@V?$_List_val@U?$_List_simple_types@V?$basic_string@DU?$char_traits@D@std@@V?$allocator@D@2@@std@@@std@@@std@@@0@AAV10@@Z 00406010 f i MessageHistory.obj
 0001:00005010       ??$move@AAV?$_List_unchecked_const_iterator@V?$_List_val@U?$_List_simple_types@V?$basic_string@DU?$char_traits@D@std@@V?$allocator@D@2@@std@@@std@@@std@@U_Iterator_base0@2@@std@@@std@@YA$$QAV?$_List_unchecked_const_iterator@V?$_List_val@U?$_List_simple_types@V?$basic_string@DU?$char_traits@D@std@@V?$allocator@D@2@@std@@@std@@@std@@U_Iterator_base0@2@@0@AAV10@@Z 00406010 f i MessageHistory.obj
 0001:00005010       ??$addressof@PAU?$_List_node@V?$basic_string@DU?$char_traits@D@std@@V?$allocator@D@2@@std@@PAX@std@@@std@@YAPAPAU?$_List_node@V?$basic_string@DU?$char_traits@D@std@@V?$allocator@D@2@@std@@PAX@0@AAPAU10@@Z 00406010 f i MessageHistory.obj
 0001:00005010       ??$addressof@V?$basic_string@DU?$char_traits@D@std@@V?$allocator@D@2@@std@@@std@@YAPAV?$basic_string@DU?$char_traits@D@std@@V?$allocator@D@2@@0@AAV10@@Z 00406010 f i MessageHistory.obj
 0001:00005010       ??$forward@V?$allocator@D@std@@@std@@YA$$QAV?$allocator@D@0@AAV10@@Z 00406010 f i MessageHistory.obj
 0001:00005010       ??$addressof@V?$_String_val@U?$_Simple_types@D@std@@@std@@@std@@YAPAV?$_String_val@U?$_Simple_types@D@std@@@0@AAV10@@Z 00406010 f i MessageHistory.obj
 0001:00005010       ??$_Unfancy@D@std@@YAPADPAD@Z 00406010 f i MessageHistory.obj
 0001:00005010       ??$move@AAV?$basic_string@DU?$char_traits@D@std@@V?$allocator@D@2@@std@@@std@@YA$$QAV?$basic_string@DU?$char_traits@D@std@@V?$allocator@D@2@@0@AAV10@@Z 00406010 f i MessageHistory.obj
 0001:00005010       ??$forward@ABQAD@std@@YAABQADABQAD@Z 00406010 f i MessageHistory.obj
 0001:00005010       ??$addressof@$$CBV?$_String_val@U?$_Simple_types@D@std@@@std@@@std@@YAPBV?$_String_val@U?$_Simple_types@D@std@@@0@ABV10@@Z 00406010 f i MessageHistory.obj
 0001:00005010       ??$addressof@V?$_List_val@U?$_List_simple_types@V?$basic_string@DU?$char_traits@D@std@@V?$allocator@D@2@@std@@@std@@@std@@@std@@YAPAV?$_List_val@U?$_List_simple_types@V?$basic_string@DU?$char_traits@D@std@@V?$allocator@D@2@@std@@@std@@@0@AAV10@@Z 00406010 f i MessageHistory.obj
 0001:00005010       ??$forward@V?$basic_string@DU?$char_traits@D@std@@V?$allocator@D@2@@std@@@std@@YA$$QAV?$basic_string@DU?$char_traits@D@std@@V?$allocator@D@2@@0@AAV10@@Z 00406010 f i MessageHistory.obj
 0001:00005010       ??$move@AAV?$allocator@D@std@@@std@@YA$$QAV?$allocator@D@0@AAV10@@Z 00406010 f i MessageHistory.obj
 0001:00005020       ??$_Deallocate@$07$0A@@std@@YAXPAXI@Z 00406020 f i MessageHistory.obj
 0001:00005080       ??$_Emplace@V?$basic_string@DU?$char_traits@D@std@@V?$allocator@D@2@@std@@@?$list@V?$basic_string@DU?$char_traits@D@std@@V?$allocator@D@2@@std@@V?$allocator@V?$basic_string@DU?$char_traits@D@std@@V?$allocator@D@2@@std@@@2@@std@@QAEPAU?$_List_node@V?$basic_string@DU?$char_traits@D@std@@V?$allocator@D@2@@std@@PAX@1@QAU21@$$QAV?$basic_string@DU?$char_traits@D@std@@V?$allocator@D@2@@1@@Z 00406080 f i MessageHistory.obj
 0001:00005110       ??$_Free_non_head@V?$allocator@U?$_List_node@V?$basic_string@DU?$char_traits@D@std@@V?$allocator@D@2@@std@@PAX@std@@@std@@@?$_List_node@V?$basic_string@DU?$char_traits@D@std@@V?$allocator@D@2@@std@@PAX@std@@SAXAAV?$allocator@U?$_List_node@V?$basic_string@DU?$char_traits@D@std@@V?$allocator@D@2@@std@@PAX@std@@@1@PAU01@@Z 00406110 f i MessageHistory.obj
 0001:00005160       ??$_Freenode0@V?$allocator@U?$_List_node@V?$basic_string@DU?$char_traits@D@std@@V?$allocator@D@2@@std@@PAX@std@@@std@@@?$_List_node@V?$basic_string@DU?$char_traits@D@std@@V?$allocator@D@2@@std@@PAX@std@@SAXAAV?$allocator@U?$_List_node@V?$basic_string@DU?$char_traits@D@std@@V?$allocator@D@2@@std@@PAX@std@@@1@PAU01@@Z 00406160 f i MessageHistory.obj
 0001:000051d0       ??$_Freenode@V?$allocator@U?$_List_node@V?$basic_string@DU?$char_traits@D@std@@V?$allocator@D@2@@std@@PAX@std@@@std@@@?$_List_node@V?$basic_string@DU?$char_traits@D@std@@V?$allocator@D@2@@std@@PAX@std@@SAXAAV?$allocator@U?$_List_node@V?$basic_string@DU?$char_traits@D@std@@V?$allocator@D@2@@std@@PAX@std@@@1@PAU01@@Z 004061d0 f i MessageHistory.obj
 0001:00005240       ??$_Get_size_of_n@$00@std@@YAII@Z 00406240 f i MessageHistory.obj
 0001:00005250       ??$_Get_size_of_n@$0CA@@std@@YAII@Z 00406250 f i MessageHistory.obj
 0001:00005280       ??$_Get_unwrapped_n@V?$_List_const_iterator@V?$_List_val@U?$_List_simple_types@V?$basic_string@DU?$char_traits@D@std@@V?$allocator@D@2@@std@@@std@@@std@@@std@@I@std@@YA?AV?$_List_unchecked_const_iterator@V?$_List_val@U?$_List_simple_types@V?$basic_string@DU?$char_traits@D@std@@V?$allocator@D@2@@std@@@std@@@std@@U_Iterator_base0@2@@0@$$QAV?$_List_const_iterator@V?$_List_val@U?$_List_simple_types@V?$basic_string@DU?$char_traits@D@std@@V?$allocator@D@2@@std@@@std@@@std@@@0@I@Z 00406280 f i MessageHistory.obj
 0001:00005280       ??$_Get_unwrapped@AAV?$_List_const_iterator@V?$_List_val@U?$_List_simple_types@V?$basic_string@DU?$char_traits@D@std@@V?$allocator@D@2@@std@@@std@@@std@@@std@@@std@@YA?AV?$_List_unchecked_const_iterator@V?$_List_val@U?$_List_simple_types@V?$basic_string@DU?$char_traits@D@std@@V?$allocator@D@2@@std@@@std@@@std@@U_Iterator_base0@2@@0@AAV?$_List_const_iterator@V?$_List_val@U?$_List_simple_types@V?$basic_string@DU?$char_traits@D@std@@V?$allocator@D@2@@std@@@std@@@std@@@0@@Z 00406280 f i MessageHistory.obj
 0001:000052a0       ??$_Reallocate_for@V<lambda_9366063389c5f42a00a5088cf24e69de>@@PBD@?$basic_string@DU?$char_traits@D@std@@V?$allocator@D@2@@std@@AAEAAV01@IV<lambda_9366063389c5f42a00a5088cf24e69de>@@PBD@Z 004062a0 f i MessageHistory.obj
 0001:00005370       ??$_Seek_wrapped@V?$_List_const_iterator@V?$_List_val@U?$_List_simple_types@V?$basic_string@DU?$char_traits@D@std@@V?$allocator@D@2@@std@@@std@@@std@@@std@@V?$_List_unchecked_const_iterator@V?$_List_val@U?$_List_simple_types@V?$basic_string@DU?$char_traits@D@std@@V?$allocator@D@2@@std@@@std@@@std@@U_Iterator_base0@2@@2@@std@@YAXAAV?$_List_const_iterator@V?$_List_val@U?$_List_simple_types@V?$basic_string@DU?$char_traits@D@std@@V?$allocator@D@2@@std@@@std@@@std@@@0@$$QAV?$_List_unchecked_const_iterator@V?$_List_val@U?$_List_simple_types@V?$basic_string@DU?$char_traits@D@std@@V?$allocator@D@2@@std@@@std@@@std@@U_Iterator_base0@2@@0@@Z 00406370 f i MessageHistory.obj
 0001:00005390       ??$advance@V?$_List_const_iterator@V?$_List_val@U?$_List_simple_types@V?$basic_string@DU?$char_traits@D@std@@V?$allocator@D@2@@std@@@std@@@std@@@std@@I@std@@YAXAAV?$_List_const_iterator@V?$_List_val@U?$_List_simple_types@V?$basic_string@DU?$char_traits@D@std@@V?$allocator@D@2@@std@@@std@@@std@@@0@I@Z 00406390 f i MessageHistory.obj
 0001:00005400       ??$construct@V?$basic_string@DU?$char_traits@D@std@@V?$allocator@D@2@@std@@V12@@?$_Default_allocator_traits@V?$allocator@U?$_List_node@V?$basic_string@DU?$char_traits@D@std@@V?$allocator@D@2@@std@@PAX@std@@@std@@@std@@SAXAAV?$allocator@U?$_List_node@V?$basic_string@DU?$char_traits@D@std@@V?$allocator@D@2@@std@@PAX@std@@@1@QAV?$basic_string@DU?$char_traits@D@std@@V?$allocator@D@2@@1@$$QAV31@@Z 00406400 f i MessageHistory.obj
 0001:00005430       ??$destroy@V?$basic_string@DU?$char_traits@D@std@@V?$allocator@D@2@@std@@@?$_Default_allocator_traits@V?$allocator@U?$_List_node@V?$basic_string@DU?$char_traits@D@std@@V?$allocator@D@2@@std@@PAX@std@@@std@@@std@@SAXAAV?$allocator@U?$_List_node@V?$basic_string@DU?$char_traits@D@std@@V?$allocator@D@2@@std@@PAX@std@@@1@QAV?$basic_string@DU?$char_traits@D@std@@V?$allocator@D@2@@1@@Z 00406430 f i MessageHistory.obj
 0001:00005440       ??$distance@V?$_List_const_iterator@V?$_List_val@U?$_List_simple_types@V?$basic_string@DU?$char_traits@D@std@@V?$allocator@D@2@@std@@@std@@@std@@@std@@@std@@YAHV?$_List_const_iterator@V?$_List_val@U?$_List_simple_types@V?$basic_string@DU?$char_traits@D@std@@V?$allocator@D@2@@std@@@std@@@std@@@0@0@Z 00406440 f i MessageHistory.obj
 0001:000054b0       ??$max@I@std@@YAABIABI0@Z  004064b0 f i MessageHistory.obj
 0001:000054e0       ??$min@I@std@@YAABIABI0@Z  004064e0 f i MessageHistory.obj
 0001:00005510       ??0?$_Alloc_construct_ptr@V?$allocator@U?$_List_node@V?$basic_string@DU?$char_traits@D@std@@V?$allocator@D@2@@std@@PAX@std@@@std@@@std@@QAE@AAV?$allocator@U?$_List_node@V?$basic_string@DU?$char_traits@D@std@@V?$allocator@D@2@@std@@PAX@std@@@1@@Z 00406510 f i MessageHistory.obj
 0001:00005540       ??0?$_List_const_iterator@V?$_List_val@U?$_List_simple_types@V?$basic_string@DU?$char_traits@D@std@@V?$allocator@D@2@@std@@@std@@@std@@@std@@QAE@PAU?$_List_node@V?$basic_string@DU?$char_traits@D@std@@V?$allocator@D@2@@std@@PAX@1@PBV?$_List_val@U?$_List_simple_types@V?$basic_string@DU?$char_traits@D@std@@V?$allocator@D@2@@std@@@std@@@1@@Z 00406540 f i MessageHistory.obj
 0001:00005560       ??0?$_List_iterator@V?$_List_val@U?$_List_simple_types@V?$basic_string@DU?$char_traits@D@std@@V?$allocator@D@2@@std@@@std@@@std@@@std@@QAE@PAU?$_List_node@V?$basic_string@DU?$char_traits@D@std@@V?$allocator@D@2@@std@@PAX@1@PBV?$_List_val@U?$_List_simple_types@V?$basic_string@DU?$char_traits@D@std@@V?$allocator@D@2@@std@@@std@@@1@@Z 00406560 f i MessageHistory.obj
 0001:00005580       ??0?$_List_unchecked_const_iterator@V?$_List_val@U?$_List_simple_types@V?$basic_string@DU?$char_traits@D@std@@V?$allocator@D@2@@std@@@std@@@std@@U_Iterator_base0@2@@std@@QAE@PAU?$_List_node@V?$basic_string@DU?$char_traits@D@std@@V?$allocator@D@2@@std@@PAX@1@PBV?$_List_val@U?$_List_simple_types@V?$basic_string@DU?$char_traits@D@std@@V?$allocator@D@2@@std@@@std@@@1@@Z 00406580 f i MessageHistory.obj
 0001:000055b0       ??0?$_String_val@U?$_Simple_types@D@std@@@std@@QAE@XZ 004065b0 f i MessageHistory.obj
 0001:000055e0       ?_Get_first@?$_Compressed_pair@V?$allocator@U?$_List_node@V?$basic_string@DU?$char_traits@D@std@@V?$allocator@D@2@@std@@PAX@std@@@std@@V?$_List_val@U?$_List_simple_types@V?$basic_string@DU?$char_traits@D@std@@V?$allocator@D@2@@std@@@std@@@2@$00@std@@QBEABV?$allocator@U?$_List_node@V?$basic_string@DU?$char_traits@D@std@@V?$allocator@D@2@@std@@PAX@std@@@2@XZ 004065e0 f i MessageHistory.obj
 0001:000055e0       ??0_Bxty@?$_String_val@U?$_Simple_types@D@std@@@std@@QAE@XZ 004065e0 f i MessageHistory.obj
 0001:000055e0       ?_Get_first@?$_Compressed_pair@V?$allocator@D@std@@V?$_String_val@U?$_Simple_types@D@std@@@2@$00@std@@QAEAAV?$allocator@D@2@XZ 004065e0 f i MessageHistory.obj
 0001:000055e0       ??0?$allocator@D@std@@QAE@XZ 004065e0 f i MessageHistory.obj
 0001:000055e0       ?_Get_first@?$_Compressed_pair@V?$allocator@U?$_List_node@V?$basic_string@DU?$char_traits@D@std@@V?$allocator@D@2@@std@@PAX@std@@@std@@V?$_List_val@U?$_List_simple_types@V?$basic_string@DU?$char_traits@D@std@@V?$allocator@D@2@@std@@@std@@@2@$00@std@@QAEAAV?$allocator@U?$_List_node@V?$basic_string@DU?$char_traits@D@std@@V?$allocator@D@2@@std@@PAX@std@@@2@XZ 004065e0 f i MessageHistory.obj
 0001:000055e0       ??0?$allocator@U?$_List_node@V?$basic_string@DU?$char_traits@D@std@@V?$allocator@D@2@@std@@PAX@std@@@std@@QAE@XZ 004065e0 f i jaccessinspector.obj
 0001:000055e0       ?_Get_first@?$_Compressed_pair@V?$allocator@D@std@@V?$_String_val@U?$_Simple_types@D@std@@@2@$00@std@@QBEABV?$allocator@D@2@XZ 004065e0 f i MessageHistory.obj
 0001:000055f0       ??0?$basic_string@DU?$char_traits@D@std@@V?$allocator@D@2@@std@@QAE@$$QAV01@@Z 004065f0 f i MessageHistory.obj
 0001:00005680       ??0?$basic_string@DU?$char_traits@D@std@@V?$allocator@D@2@@std@@QAE@QBD@Z 00406680 f i MessageHistory.obj
 0001:00005710       ??0_Fake_proxy_ptr_impl@std@@QAE@ABU_Fake_allocator@1@ABU_Container_base0@1@@Z 00406710 f i MessageHistory.obj
 0001:00005720       ??0bad_alloc@std@@AAE@QBD@Z 00406720 f i MessageHistory.obj
 0001:00005750       ??0bad_alloc@std@@QAE@ABV01@@Z 00406750 f i MessageHistory.obj
 0001:00005780       ??0bad_array_new_length@std@@QAE@ABV01@@Z 00406780 f i MessageHistory.obj
 0001:000057b0       ??0bad_array_new_length@std@@QAE@XZ 004067b0 f i MessageHistory.obj
 0001:000057e0       ??0exception@std@@QAE@ABV01@@Z 004067e0 f i MessageHistory.obj
 0001:00005820       ??0exception@std@@QAE@QBDH@Z 00406820 f i MessageHistory.obj
 0001:00005850       ??1?$_Alloc_construct_ptr@V?$allocator@U?$_List_node@V?$basic_string@DU?$char_traits@D@std@@V?$allocator@D@2@@std@@PAX@std@@@std@@@std@@QAE@XZ 00406850 f i MessageHistory.obj
 0001:000058b0       ??1?$_Compressed_pair@V?$allocator@D@std@@V?$_String_val@U?$_Simple_types@D@std@@@2@$00@std@@QAE@XZ 004068b0 f i MessageHistory.obj
 0001:000058d0       ??1?$_List_node_emplace_op2@V?$allocator@U?$_List_node@V?$basic_string@DU?$char_traits@D@std@@V?$allocator@D@2@@std@@PAX@std@@@std@@@std@@QAE@XZ 004068d0 f i MessageHistory.obj
 0001:00005940       ??1?$_String_val@U?$_Simple_types@D@std@@@std@@QAE@XZ 00406940 f i MessageHistory.obj
 0001:00005960       ??1?$basic_string@DU?$char_traits@D@std@@V?$allocator@D@2@@std@@QAE@XZ 00406960 f i MessageHistory.obj
 0001:00005980       ?_Orphan_all@_Container_base0@std@@QAEXXZ 00406980 f i MessageHistory.obj
 0001:00005980       ?_Orphan_non_end@?$_List_val@U?$_List_simple_types@V?$basic_string@DU?$char_traits@D@std@@V?$allocator@D@2@@std@@@std@@@std@@QAEXXZ 00406980 f i MessageHistory.obj
 0001:00005980       ??1_Bxty@?$_String_val@U?$_Simple_types@D@std@@@std@@QAE@XZ 00406980 f i MessageHistory.obj
 0001:00005980       ?_Release@_Fake_proxy_ptr_impl@std@@QAEXXZ 00406980 f i MessageHistory.obj
 0001:00005990       ??1bad_alloc@std@@UAE@XZ   00406990 f i MessageHistory.obj
 0001:000059b0       ??1bad_array_new_length@std@@UAE@XZ 004069b0 f i MessageHistory.obj
 0001:000059d0       ??1exception@std@@UAE@XZ   004069d0 f i MessageHistory.obj
 0001:00005a00       ??2@YAPAXIPAX@Z            00406a00 f i MessageHistory.obj
 0001:00005a10       ??8?$_List_const_iterator@V?$_List_val@U?$_List_simple_types@V?$basic_string@DU?$char_traits@D@std@@V?$allocator@D@2@@std@@@std@@@std@@@std@@QBE_NABV01@@Z 00406a10 f i MessageHistory.obj
 0001:00005a10       ??8?$_List_unchecked_const_iterator@V?$_List_val@U?$_List_simple_types@V?$basic_string@DU?$char_traits@D@std@@V?$allocator@D@2@@std@@@std@@@std@@U_Iterator_base0@2@@std@@QBE_NABV01@@Z 00406a10 f i MessageHistory.obj
 0001:00005a40       ??9?$_List_unchecked_const_iterator@V?$_List_val@U?$_List_simple_types@V?$basic_string@DU?$char_traits@D@std@@V?$allocator@D@2@@std@@@std@@@std@@U_Iterator_base0@2@@std@@QBE_NABV01@@Z 00406a40 f i MessageHistory.obj
 0001:00005a40       ??9?$_List_const_iterator@V?$_List_val@U?$_List_simple_types@V?$basic_string@DU?$char_traits@D@std@@V?$allocator@D@2@@std@@@std@@@std@@@std@@QBE_NABV01@@Z 00406a40 f i MessageHistory.obj
 0001:00005a80       ??D?$_List_const_iterator@V?$_List_val@U?$_List_simple_types@V?$basic_string@DU?$char_traits@D@std@@V?$allocator@D@2@@std@@@std@@@std@@@std@@QBEABV?$basic_string@DU?$char_traits@D@std@@V?$allocator@D@2@@1@XZ 00406a80 f i MessageHistory.obj
 0001:00005aa0       ??E?$_List_unchecked_const_iterator@V?$_List_val@U?$_List_simple_types@V?$basic_string@DU?$char_traits@D@std@@V?$allocator@D@2@@std@@@std@@@std@@U_Iterator_base0@2@@std@@QAEAAV01@XZ 00406aa0 f i MessageHistory.obj
 0001:00005aa0       ??E?$_List_const_iterator@V?$_List_val@U?$_List_simple_types@V?$basic_string@DU?$char_traits@D@std@@V?$allocator@D@2@@std@@@std@@@std@@@std@@QAEAAV01@XZ 00406aa0 f i MessageHistory.obj
 0001:00005ac0       ??F?$_List_const_iterator@V?$_List_val@U?$_List_simple_types@V?$basic_string@DU?$char_traits@D@std@@V?$allocator@D@2@@std@@@std@@@std@@@std@@QAEAAV01@XZ 00406ac0 f i MessageHistory.obj
 0001:00005af0       ??R<lambda_9366063389c5f42a00a5088cf24e69de>@@QBEXQADIQBD@Z 00406af0 f i MessageHistory.obj
 0001:00005b30       ??_G?$basic_string@DU?$char_traits@D@std@@V?$allocator@D@2@@std@@QAEPAXI@Z 00406b30 f i MessageHistory.obj
 0001:00005b60       ??_Gbad_alloc@std@@UAEPAXI@Z 00406b60 f i MessageHistory.obj
 0001:00005b60       ??_Ebad_alloc@std@@UAEPAXI@Z 00406b60 f i MessageHistory.obj
 0001:00005b90       ??_Gbad_array_new_length@std@@UAEPAXI@Z 00406b90 f i MessageHistory.obj
 0001:00005b90       ??_Ebad_array_new_length@std@@UAEPAXI@Z 00406b90 f i MessageHistory.obj
 0001:00005bc0       ??_Gexception@std@@UAEPAXI@Z 00406bc0 f i MessageHistory.obj
 0001:00005bc0       ??_Eexception@std@@UAEPAXI@Z 00406bc0 f i MessageHistory.obj
 0001:00005bf0       ?_Adjust_manually_vector_aligned@std@@YAXAAPAXAAI@Z 00406bf0 f i MessageHistory.obj
 0001:00005c60       ?_Adopt@_Iterator_base0@std@@QAEXPBX@Z 00406c60 f i MessageHistory.obj
 0001:00005c60       ?_Alloc_proxy@_Container_base0@std@@QAEXABU_Fake_allocator@2@@Z 00406c60 f i MessageHistory.obj
 0001:00005c60       ?_Orphan_ptr2@?$_List_val@U?$_List_simple_types@V?$basic_string@DU?$char_traits@D@std@@V?$allocator@D@2@@std@@@std@@@std@@QAEXPAU?$_List_node@V?$basic_string@DU?$char_traits@D@std@@V?$allocator@D@2@@std@@PAX@2@@Z 00406c60 f i MessageHistory.obj
 0001:00005c70       ?_Allocate@?$_Alloc_construct_ptr@V?$allocator@U?$_List_node@V?$basic_string@DU?$char_traits@D@std@@V?$allocator@D@2@@std@@PAX@std@@@std@@@std@@QAEXXZ 00406c70 f i MessageHistory.obj
 0001:00005ca0       ?_Allocate@_Default_allocate_traits@std@@SAPAXI@Z 00406ca0 f i MessageHistory.obj
 0001:00005cc0       ?_Calculate_growth@?$basic_string@DU?$char_traits@D@std@@V?$allocator@D@2@@std@@ABEII@Z 00406cc0 f i MessageHistory.obj
 0001:00005cf0       ?_Calculate_growth@?$basic_string@DU?$char_traits@D@std@@V?$allocator@D@2@@std@@CAIIII@Z 00406cf0 f i MessageHistory.obj
 0001:00005d50       ?_Getal@?$basic_string@DU?$char_traits@D@std@@V?$allocator@D@2@@std@@ABEABV?$allocator@D@2@XZ 00406d50 f i MessageHistory.obj
 0001:00005d50       ?_Getal@?$list@V?$basic_string@DU?$char_traits@D@std@@V?$allocator@D@2@@std@@V?$allocator@V?$basic_string@DU?$char_traits@D@std@@V?$allocator@D@2@@std@@@2@@std@@ABEABV?$allocator@U?$_List_node@V?$basic_string@DU?$char_traits@D@std@@V?$allocator@D@2@@std@@PAX@std@@@2@XZ 00406d50 f i MessageHistory.obj
 0001:00005d50       ?_Getal@?$list@V?$basic_string@DU?$char_traits@D@std@@V?$allocator@D@2@@std@@V?$allocator@V?$basic_string@DU?$char_traits@D@std@@V?$allocator@D@2@@std@@@2@@std@@AAEAAV?$allocator@U?$_List_node@V?$basic_string@DU?$char_traits@D@std@@V?$allocator@D@2@@std@@PAX@std@@@2@XZ 00406d50 f i MessageHistory.obj
 0001:00005d50       ?_Getal@?$basic_string@DU?$char_traits@D@std@@V?$allocator@D@2@@std@@AAEAAV?$allocator@D@2@XZ 00406d50 f i MessageHistory.obj
 0001:00005d70       ?_Getcont@_Iterator_base0@std@@QBEPBU_Container_base0@2@XZ 00406d70 f i MessageHistory.obj
 0001:00005d80       ?_Large_string_engaged@?$_String_val@U?$_Simple_types@D@std@@@std@@QBE_NXZ 00406d80 f i MessageHistory.obj
 0001:00005db0       ?_Memcpy_val_from@?$basic_string@DU?$char_traits@D@std@@V?$allocator@D@2@@std@@AAEXABV12@@Z 00406db0 f i MessageHistory.obj
 0001:00005df0       ?_Myptr@?$_String_val@U?$_Simple_types@D@std@@@std@@QBEPBDXZ 00406df0 f i MessageHistory.obj
 0001:00005df0       ?_Myptr@?$_String_val@U?$_Simple_types@D@std@@@std@@QAEPADXZ 00406df0 f i MessageHistory.obj
 0001:00005e30       ?_Seek_to@?$_List_const_iterator@V?$_List_val@U?$_List_simple_types@V?$basic_string@DU?$char_traits@D@std@@V?$allocator@D@2@@std@@@std@@@std@@@std@@QAEXV?$_List_unchecked_const_iterator@V?$_List_val@U?$_List_simple_types@V?$basic_string@DU?$char_traits@D@std@@V?$allocator@D@2@@std@@@std@@@std@@U_Iterator_base0@2@@2@@Z 00406e30 f i MessageHistory.obj
 0001:00005e50       ?_Take_contents@?$basic_string@DU?$char_traits@D@std@@V?$allocator@D@2@@std@@AAEXAAV12@U?$integral_constant@_N$00@2@@Z 00406e50 f i MessageHistory.obj
 0001:00005e80       ?_Throw_bad_array_new_length@std@@YAXXZ 00406e80 f i MessageHistory.obj
 0001:00005ea0       ?_Tidy_deallocate@?$basic_string@DU?$char_traits@D@std@@V?$allocator@D@2@@std@@AAEXXZ 00406ea0 f i MessageHistory.obj
 0001:00005f60       ?_Tidy_init@?$basic_string@DU?$char_traits@D@std@@V?$allocator@D@2@@std@@AAEXXZ 00406f60 f i MessageHistory.obj
 0001:00005fa0       ?_Transfer_before@?$_List_node_emplace_op2@V?$allocator@U?$_List_node@V?$basic_string@DU?$char_traits@D@std@@V?$allocator@D@2@@std@@PAX@std@@@std@@@std@@QAEPAU?$_List_node@V?$basic_string@DU?$char_traits@D@std@@V?$allocator@D@2@@std@@PAX@2@QAU32@@Z 00406fa0 f i MessageHistory.obj
 0001:00006010       ?_Unchecked_erase@?$list@V?$basic_string@DU?$char_traits@D@std@@V?$allocator@D@2@@std@@V?$allocator@V?$basic_string@DU?$char_traits@D@std@@V?$allocator@D@2@@std@@@2@@std@@AAEPAU?$_List_node@V?$basic_string@DU?$char_traits@D@std@@V?$allocator@D@2@@std@@PAX@2@QAU32@@Z 00407010 f i MessageHistory.obj
 0001:00006080       ?_Unwrapped@?$_List_const_iterator@V?$_List_val@U?$_List_simple_types@V?$basic_string@DU?$char_traits@D@std@@V?$allocator@D@2@@std@@@std@@@std@@@std@@QBE?AV?$_List_unchecked_const_iterator@V?$_List_val@U?$_List_simple_types@V?$basic_string@DU?$char_traits@D@std@@V?$allocator@D@2@@std@@@std@@@std@@U_Iterator_base0@2@@2@XZ 00407080 f i MessageHistory.obj
 0001:000060b0       ?_Xlen_string@std@@YAXXZ   004070b0 f i MessageHistory.obj
 0001:000060c0       ?allocate@?$allocator@D@std@@QAEPADI@Z 004070c0 f i MessageHistory.obj
 0001:000060f0       ?allocate@?$allocator@U?$_List_node@V?$basic_string@DU?$char_traits@D@std@@V?$allocator@D@2@@std@@PAX@std@@@std@@QAEPAU?$_List_node@V?$basic_string@DU?$char_traits@D@std@@V?$allocator@D@2@@std@@PAX@2@I@Z 004070f0 f i MessageHistory.obj
 0001:00006120       ?assign@?$_Narrow_char_traits@DH@std@@SAXAADABD@Z 00407120 f i MessageHistory.obj
 0001:00006130       ?assign@?$basic_string@DU?$char_traits@D@std@@V?$allocator@D@2@@std@@QAEAAV12@QBD@Z 00407130 f i MessageHistory.obj
 0001:00006160       ?assign@?$basic_string@DU?$char_traits@D@std@@V?$allocator@D@2@@std@@QAEAAV12@QBDI@Z 00407160 f i MessageHistory.obj
 0001:000061e0       ?begin@?$list@V?$basic_string@DU?$char_traits@D@std@@V?$allocator@D@2@@std@@V?$allocator@V?$basic_string@DU?$char_traits@D@std@@V?$allocator@D@2@@std@@@2@@std@@QAE?AV?$_List_iterator@V?$_List_val@U?$_List_simple_types@V?$basic_string@DU?$char_traits@D@std@@V?$allocator@D@2@@std@@@std@@@std@@@2@XZ 004071e0 f i MessageHistory.obj
 0001:00006210       ?c_str@?$basic_string@DU?$char_traits@D@std@@V?$allocator@D@2@@std@@QBEPBDXZ 00407210 f i MessageHistory.obj
 0001:00006230       ?clear@?$list@V?$basic_string@DU?$char_traits@D@std@@V?$allocator@D@2@@std@@V?$allocator@V?$basic_string@DU?$char_traits@D@std@@V?$allocator@D@2@@std@@@2@@std@@QAEXXZ 00407230 f i MessageHistory.obj
 0001:00006290       ?copy@?$_Narrow_char_traits@DH@std@@SAPADQADQBDI@Z 00407290 f i MessageHistory.obj
 0001:000062b0       ?deallocate@?$_Default_allocator_traits@V?$allocator@U?$_List_node@V?$basic_string@DU?$char_traits@D@std@@V?$allocator@D@2@@std@@PAX@std@@@std@@@std@@SAXAAV?$allocator@U?$_List_node@V?$basic_string@DU?$char_traits@D@std@@V?$allocator@D@2@@std@@PAX@std@@@2@QAU?$_List_node@V?$basic_string@DU?$char_traits@D@std@@V?$allocator@D@2@@std@@PAX@2@I@Z 004072b0 f i MessageHistory.obj
 0001:000062d0       ?deallocate@?$allocator@D@std@@QAEXQADI@Z 004072d0 f i MessageHistory.obj
 0001:000062f0       ?deallocate@?$allocator@U?$_List_node@V?$basic_string@DU?$char_traits@D@std@@V?$allocator@D@2@@std@@PAX@std@@@std@@QAEXQAU?$_List_node@V?$basic_string@DU?$char_traits@D@std@@V?$allocator@D@2@@std@@PAX@2@I@Z 004072f0 f i MessageHistory.obj
 0001:00006310       ?empty@?$list@V?$basic_string@DU?$char_traits@D@std@@V?$allocator@D@2@@std@@V?$allocator@V?$basic_string@DU?$char_traits@D@std@@V?$allocator@D@2@@std@@@2@@std@@QBE_NXZ 00407310 f i MessageHistory.obj
 0001:00006340       ?end@?$list@V?$basic_string@DU?$char_traits@D@std@@V?$allocator@D@2@@std@@V?$allocator@V?$basic_string@DU?$char_traits@D@std@@V?$allocator@D@2@@std@@@2@@std@@QAE?AV?$_List_iterator@V?$_List_val@U?$_List_simple_types@V?$basic_string@DU?$char_traits@D@std@@V?$allocator@D@2@@std@@@std@@@std@@@2@XZ 00407340 f i MessageHistory.obj
 0001:00006370       ?length@?$_Narrow_char_traits@DH@std@@SAIQBD@Z 00407370 f i MessageHistory.obj
 0001:00006390       ?max@?$numeric_limits@H@std@@SAHXZ 00407390 f i MessageHistory.obj
 0001:000063a0       ?max_size@?$_Default_allocator_traits@V?$allocator@D@std@@@std@@SAIABV?$allocator@D@2@@Z 004073a0 f i MessageHistory.obj
 0001:000063b0       ?max_size@?$_Default_allocator_traits@V?$allocator@U?$_List_node@V?$basic_string@DU?$char_traits@D@std@@V?$allocator@D@2@@std@@PAX@std@@@std@@@std@@SAIABV?$allocator@U?$_List_node@V?$basic_string@DU?$char_traits@D@std@@V?$allocator@D@2@@std@@PAX@std@@@2@@Z 004073b0 f i MessageHistory.obj
 0001:000063c0       ?max_size@?$basic_string@DU?$char_traits@D@std@@V?$allocator@D@2@@std@@QBEIXZ 004073c0 f i MessageHistory.obj
 0001:00006420       ?max_size@?$list@V?$basic_string@DU?$char_traits@D@std@@V?$allocator@D@2@@std@@V?$allocator@V?$basic_string@DU?$char_traits@D@std@@V?$allocator@D@2@@std@@@2@@std@@QBEIXZ 00407420 f i MessageHistory.obj
 0001:00006460       ?move@?$_Narrow_char_traits@DH@std@@SAPADQADQBDI@Z 00407460 f i MessageHistory.obj
 0001:00006480       ?pop_front@?$list@V?$basic_string@DU?$char_traits@D@std@@V?$allocator@D@2@@std@@V?$allocator@V?$basic_string@DU?$char_traits@D@std@@V?$allocator@D@2@@std@@@2@@std@@QAEXXZ 00407480 f i MessageHistory.obj
 0001:000064a0       ?push_back@?$list@V?$basic_string@DU?$char_traits@D@std@@V?$allocator@D@2@@std@@V?$allocator@V?$basic_string@DU?$char_traits@D@std@@V?$allocator@D@2@@std@@@2@@std@@QAEX$$QAV?$basic_string@DU?$char_traits@D@std@@V?$allocator@D@2@@2@@Z 004074a0 f i MessageHistory.obj
 0001:000064d0       ?size@?$list@V?$basic_string@DU?$char_traits@D@std@@V?$allocator@D@2@@std@@V?$allocator@V?$basic_string@DU?$char_traits@D@std@@V?$allocator@D@2@@std@@@2@@std@@QBEIXZ 004074d0 f i MessageHistory.obj
 0001:000064f0       ?what@exception@std@@UBEPBDXZ 004074f0 f i MessageHistory.obj
 0001:00006540       _WinMain@16                00407540 f   jaccessinspector.obj
 0001:00006690       ?TimerProc@@YGXPAUHWND__@@IIK@Z 00407690 f   jaccessinspector.obj
 0001:000066d0       ?KeyboardProc@@YGJHIJ@Z    004076d0 f   jaccessinspector.obj
 0001:00006770       ?MouseProc@@YGJHIJ@Z       00407770 f   jaccessinspector.obj
 0001:000067d0       ?InitWindow@@YAHPAX@Z      004077d0 f   jaccessinspector.obj
 0001:00006870       ?jaccessinspectorDialogProc@@YGHPAUHWND__@@IIJ@Z 00407870 f   jaccessinspector.obj
 0001:000082e0       ?HandleJavaShutdown@@YAXJ@Z 004092e0 f   jaccessinspector.obj
 0001:00008350       ?HandleJavaFocusGained@@YAXJPAV_jobject@@0@Z 00409350 f   jaccessinspector.obj
 0001:000083d0       ?HandleJavaFocusLost@@YAXJPAV_jobject@@0@Z 004093d0 f   jaccessinspector.obj
 0001:00008450       ?HandleJavaCaretUpdate@@YAXJPAV_jobject@@0@Z 00409450 f   jaccessinspector.obj
 0001:00008490       ?HandleMouseClicked@@YAXJPAV_jobject@@0@Z 00409490 f   jaccessinspector.obj
 0001:000084d0       ?HandleMouseEntered@@YAXJPAV_jobject@@0@Z 004094d0 f   jaccessinspector.obj
 0001:00008510       ?HandleMouseExited@@YAXJPAV_jobject@@0@Z 00409510 f   jaccessinspector.obj
 0001:00008550       ?HandleMousePressed@@YAXJPAV_jobject@@0@Z 00409550 f   jaccessinspector.obj
 0001:00008590       ?HandleMouseReleased@@YAXJPAV_jobject@@0@Z 00409590 f   jaccessinspector.obj
 0001:000085d0       ?HandleMenuCanceled@@YAXJPAV_jobject@@0@Z 004095d0 f   jaccessinspector.obj
 0001:00008610       ?HandleMenuDeselected@@YAXJPAV_jobject@@0@Z 00409610 f   jaccessinspector.obj
 0001:00008650       ?HandleMenuSelected@@YAXJPAV_jobject@@0@Z 00409650 f   jaccessinspector.obj
 0001:00008690       ?HandlePopupMenuCanceled@@YAXJPAV_jobject@@0@Z 00409690 f   jaccessinspector.obj
 0001:000086d0       ?HandlePopupMenuWillBecomeInvisible@@YAXJPAV_jobject@@0@Z 004096d0 f   jaccessinspector.obj
 0001:00008710       ?HandlePopupMenuWillBecomeVisible@@YAXJPAV_jobject@@0@Z 00409710 f   jaccessinspector.obj
 0001:00008750       ?HandlePropertyNameChange@@YAXJPAV_jobject@@0PAG1@Z 00409750 f   jaccessinspector.obj
 0001:000087d0       ?HandlePropertyDescriptionChange@@YAXJPAV_jobject@@0PAG1@Z 004097d0 f   jaccessinspector.obj
 0001:00008850       ?HandlePropertyStateChange@@YAXJPAV_jobject@@0PAG1@Z 00409850 f   jaccessinspector.obj
 0001:000088d0       ?HandlePropertyValueChange@@YAXJPAV_jobject@@0PAG1@Z 004098d0 f   jaccessinspector.obj
 0001:00008950       ?HandlePropertySelectionChange@@YAXJPAV_jobject@@0@Z 00409950 f   jaccessinspector.obj
 0001:00008990       ?HandlePropertyTextChange@@YAXJPAV_jobject@@0@Z 00409990 f   jaccessinspector.obj
 0001:000089d0       ?HandlePropertyCaretChange@@YAXJPAV_jobject@@0HH@Z 004099d0 f   jaccessinspector.obj
 0001:00008a50       ?HandlePropertyVisibleDataChange@@YAXJPAV_jobject@@0@Z 00409a50 f   jaccessinspector.obj
 0001:00008a90       ?HandlePropertyChildChange@@YAXJPAV_jobject@@000@Z 00409a90 f   jaccessinspector.obj
 0001:00008c40       ?HandlePropertyActiveDescendentChange@@YAXJPAV_jobject@@000@Z 00409c40 f   jaccessinspector.obj
 0001:00008ce0       ?HandlePropertyTableModelChange@@YAXJPAV_jobject@@0PAG1@Z 00409ce0 f   jaccessinspector.obj
 0001:00008d60       ?SaveActiveEventOptionsToRegistry@@YAHXZ 00409d60 f   jaccessinspector.obj
 0001:00009270       ?ReadActiveEventOptionsFromRegistry@@YAHXZ 0040a270 f   jaccessinspector.obj
 0001:00009c70       ?ApplyEventOptions@@YAXPAUHWND__@@@Z 0040ac70 f   jaccessinspector.obj
 0001:0000a390       ?EnableDlgItem@@YAHPAUHWND__@@HH@Z 0040b390 f   jaccessinspector.obj
 0001:0000a3d0       ?EnableMessageNavButtons@@YAXXZ 0040b3d0 f   jaccessinspector.obj
 0001:0000a650       ?AddToMessageHistory@@YGXPBD@Z 0040b650 f   jaccessinspector.obj
 0001:0000a670       ?UpdateMessageNumber@@YAHXZ 0040b670 f   jaccessinspector.obj
 0001:0000a720       ?GoToMessageDialogProc@@YGHPAUHWND__@@IIJ@Z 0040b720 f   jaccessinspector.obj
 0001:0000a9a0       ?InitGoToMessageDialogBox@@YAHPAX@Z 0040b9a0 f   jaccessinspector.obj
 0001:0000a9f0       ?ShouldCheckMonitorTheSameEventsAsJAWS@@YAHXZ 0040b9f0 f   jaccessinspector.obj
 0001:0000ab20       ?MaybeCheckMonitorTheSameEventsAsJAWS@@YAXPAUHMENU__@@@Z 0040bb20 f   jaccessinspector.obj
 0001:0000ab60       ?ShouldCheckMonitorAllEvents@@YAHXZ 0040bb60 f   jaccessinspector.obj
 0001:0000ac90       ?MaybeCheckMonitorAllEvents@@YAXPAUHMENU__@@@Z 0040bc90 f   jaccessinspector.obj
 0001:0000acd0       ?displayAccessibleInfo@@YAXJPAV_jobject@@HH@Z 0040bcd0 f   jaccessinspector.obj
 0001:0000ad40       ?displayJavaEvent@@YAXJPAV_jobject@@PAD@Z 0040bd40 f   jaccessinspector.obj
 0001:0000adf0       ?displayAccessiblePropertyChange@@YAXJPAV_jobject@@PAD@Z 0040bdf0 f   jaccessinspector.obj
 0001:0000aea0       ?echoMouseObject@@YAXXZ    0040bea0 f   jaccessinspector.obj
 0001:0000af50       ?echoMouseHWNDObject@@YAXXZ 0040bf50 f   jaccessinspector.obj
 0001:0000afc0       ?displayFocusedObject@@YAXXZ 0040bfc0 f   jaccessinspector.obj
 0001:0000b040       ?exitjaccessinspector@@YAXPAUHWND__@@@Z 0040c040 f   jaccessinspector.obj
 0001:0000b060       ?reinstallEventListeners@@YAXXZ 0040c060 f   jaccessinspector.obj
 0001:0000b2b0       ??$?0$$V@?$_Compressed_pair@V?$allocator@U?$_List_node@V?$basic_string@DU?$char_traits@D@std@@V?$allocator@D@2@@std@@PAX@std@@@std@@V?$_List_val@U?$_List_simple_types@V?$basic_string@DU?$char_traits@D@std@@V?$allocator@D@2@@std@@@std@@@2@$00@std@@QAE@U_Zero_then_variadic_args_t@1@@Z 0040c2b0 f i jaccessinspector.obj
 0001:0000b2d0       ??0?$_List_const_iterator@V?$_List_val@U?$_List_simple_types@V?$basic_string@DU?$char_traits@D@std@@V?$allocator@D@2@@std@@@std@@@std@@@std@@QAE@XZ 0040c2d0 f i jaccessinspector.obj
 0001:0000b2f0       ??0?$_List_unchecked_const_iterator@V?$_List_val@U?$_List_simple_types@V?$basic_string@DU?$char_traits@D@std@@V?$allocator@D@2@@std@@@std@@@std@@U_Iterator_base0@2@@std@@QAE@XZ 0040c2f0 f i jaccessinspector.obj
 0001:0000b310       ??0?$_List_val@U?$_List_simple_types@V?$basic_string@DU?$char_traits@D@std@@V?$allocator@D@2@@std@@@std@@@std@@QAE@XZ 0040c310 f i jaccessinspector.obj
 0001:0000b340       ??0?$list@V?$basic_string@DU?$char_traits@D@std@@V?$allocator@D@2@@std@@V?$allocator@V?$basic_string@DU?$char_traits@D@std@@V?$allocator@D@2@@std@@@2@@std@@QAE@XZ 0040c340 f i jaccessinspector.obj
 0001:0000b370       ??0MessageHistory@@QAE@XZ  0040c370 f i jaccessinspector.obj
 0001:0000b3a0       ??1?$list@V?$basic_string@DU?$char_traits@D@std@@V?$allocator@D@2@@std@@V?$allocator@V?$basic_string@DU?$char_traits@D@std@@V?$allocator@D@2@@std@@@2@@std@@QAE@XZ 0040c3a0 f i jaccessinspector.obj
 0001:0000b3c0       ??1MessageHistory@@QAE@XZ  0040c3c0 f i jaccessinspector.obj
 0001:0000b3e0       ?_Alloc_sentinel_and_proxy@?$list@V?$basic_string@DU?$char_traits@D@std@@V?$allocator@D@2@@std@@V?$allocator@V?$basic_string@DU?$char_traits@D@std@@V?$allocator@D@2@@std@@@2@@std@@AAEXXZ 0040c3e0 f i jaccessinspector.obj
 0001:0000b450       ?_Tidy@?$list@V?$basic_string@DU?$char_traits@D@std@@V?$allocator@D@2@@std@@V?$allocator@V?$basic_string@DU?$char_traits@D@std@@V?$allocator@D@2@@std@@@2@@std@@AAEXXZ 0040c450 f i jaccessinspector.obj
 0001:0000b4a0       __snprintf                 0040c4a0 f i jaccessinspector.obj
 0001:0000b4e0       __vsnprintf                0040c4e0 f i jaccessinspector.obj
 0001:0000b4ff       ??_U@YAPAXI@Z              0040c4ff f   MSVCRT:new_array.obj
 0001:0000b508       ??_V@YAXPAX@Z              0040c508 f   MSVCRT:delete_array.obj
 0001:0000b50d       ___raise_securityfailure   0040c50d f   MSVCRT:gs_report.obj
 0001:0000b535       ___report_gsfailure        0040c535 f   MSVCRT:gs_report.obj
 0001:0000b62e       ___report_rangecheckfailure 0040c62e f   MSVCRT:gs_report.obj
 0001:0000b63a       ___report_securityfailure  0040c63a f   MSVCRT:gs_report.obj
 0001:0000b710       __aulldiv                  0040c710 f   MSVCRT:ulldiv.obj
 0001:0000b778       @__security_check_cookie@4 0040c778 f   MSVCRT:secchk.obj
 0001:0000b790       __chkstk                   0040c790 f   MSVCRT:chkstk.obj
 0001:0000b790       __alloca_probe             0040c790 f   MSVCRT:chkstk.obj
 0001:0000b7bd       ??2@YAPAXI@Z               0040c7bd f   MSVCRT:new_scalar.obj
 0001:0000b7ed       ??3@YAXPAXI@Z              0040c7ed f   MSVCRT:delete_scalar_size.obj
 0001:0000b7fb       ??_Gtype_info@@UAEPAXI@Z   0040c7fb f i MSVCRT:std_type_info_static.obj
 0001:0000b7fb       ??_Etype_info@@UAEPAXI@Z   0040c7fb f i MSVCRT:std_type_info_static.obj
 0001:0000b862       ___scrt_acquire_startup_lock 0040c862 f   MSVCRT:utility.obj
 0001:0000b894       ___scrt_initialize_crt     0040c894 f   MSVCRT:utility.obj
 0001:0000b8cd       ___scrt_initialize_onexit_tables 0040c8cd f   MSVCRT:utility.obj
 0001:0000b954       ___scrt_is_nonwritable_in_current_image 0040c954 f   MSVCRT:utility.obj
 0001:0000b9e8       ___scrt_release_startup_lock 0040c9e8 f   MSVCRT:utility.obj
 0001:0000ba05       ___scrt_uninitialize_crt   0040ca05 f   MSVCRT:utility.obj
 0001:0000ba2d       __onexit                   0040ca2d f   MSVCRT:utility.obj
 0001:0000ba5a       _atexit                    0040ca5a f   MSVCRT:utility.obj
 0001:0000bb34       __Init_thread_footer       0040cb34 f   MSVCRT:thread_safe_statics.obj
 0001:0000bb7e       __Init_thread_header       0040cb7e f   MSVCRT:thread_safe_statics.obj
 0001:0000bbd0       __Init_thread_notify       0040cbd0 f   MSVCRT:thread_safe_statics.obj
 0001:0000bc06       __Init_thread_wait         0040cc06 f   MSVCRT:thread_safe_statics.obj
 0001:0000be95       _WinMainCRTStartup         0040ce95 f   MSVCRT:exe_winmain.obj
 0001:0000be9f       ??3@YAXPAX@Z               0040ce9f f   MSVCRT:delete_scalar.obj
 0001:0000bea4       ??0bad_alloc@std@@QAE@XZ   0040cea4 f i MSVCRT:throw_bad_alloc.obj
 0001:0000bebc       ?__scrt_throw_std_bad_alloc@@YAXXZ 0040cebc f   MSVCRT:throw_bad_alloc.obj
 0001:0000bed9       ?__scrt_throw_std_bad_array_new_length@@YAXXZ 0040ced9 f   MSVCRT:throw_bad_alloc.obj
 0001:0000bef6       ___isa_available_init      0040cef6 f   MSVCRT:cpu_disp.obj
 0001:0000c0c6       __get_startup_argv_mode    0040d0c6 f   MSVCRT:argv_mode.obj
 0001:0000c0ca       ___scrt_is_ucrt_dll_in_use 0040d0ca f   MSVCRT:ucrt_detection.obj
 0001:0000c0d6       ___scrt_fastfail           0040d0d6 f   MSVCRT:utility_desktop.obj
 0001:0000c1f0       ___scrt_get_show_window_mode 0040d1f0 f   MSVCRT:utility_desktop.obj
 0001:0000c221       ___scrt_initialize_mta     0040d221 f   MSVCRT:utility_desktop.obj
 0001:0000c226       __get_startup_commit_mode  0040d226 f   MSVCRT:commit_mode.obj
 0001:0000c226       ___scrt_initialize_winrt   0040d226 f   MSVCRT:utility_desktop.obj
 0001:0000c226       ___scrt_stub_for_initialize_mta 0040d226 f   MSVCRT:utility_desktop.obj
 0001:0000c226       __matherr                  0040d226 f   MSVCRT:matherr.obj
 0001:0000c226       ___scrt_exe_initialize_mta 0040d226 f   MSVCRT:utility_desktop.obj
 0001:0000c226       __get_startup_new_mode     0040d226 f   MSVCRT:new_mode.obj
 0001:0000c226       __get_startup_thread_locale_mode 0040d226 f   MSVCRT:thread_locale.obj
 0001:0000c229       ___scrt_is_managed_app     0040d229 f   MSVCRT:utility_desktop.obj
 0001:0000c26c       ___scrt_set_unhandled_exception_filter 0040d26c f   MSVCRT:utility_desktop.obj
 0001:0000c278       ___scrt_unhandled_exception_filter@4 0040d278 f   MSVCRT:utility_desktop.obj
 0001:0000c2ce       __crt_debugger_hook        0040d2ce f   MSVCRT:utility_desktop.obj
 0001:0000c2e0       __SEH_prolog4              0040d2e0 f   MSVCRT:sehprolg4.obj
 0001:0000c324       __SEH_epilog4              0040d324 f   MSVCRT:sehprolg4.obj
 0001:0000c338       __except_handler4          0040d338 f   MSVCRT:chandler4gs.obj
 0001:0000c367       __initialize_invalid_parameter_handler 0040d367 f i MSVCRT:invalid_parameter_handler.obj
 0001:0000c367       @_guard_check_icall_nop@4  0040d367 f i MSVCRT:guard_support.obj
 0001:0000c367       __initialize_denormal_control 0040d367 f i MSVCRT:denormal_control.obj
 0001:0000c3b7       ___security_init_cookie    0040d3b7 f   MSVCRT:gs_support.obj
 0001:0000c402       __get_startup_file_mode    0040d402 f   MSVCRT:file_mode.obj
 0001:0000c408       ?__scrt_initialize_type_info@@YAXXZ 0040d408 f   MSVCRT:tncleanup.obj
 0001:0000c414       __should_initialize_environment 0040d414 f   MSVCRT:env_mode.obj
 0001:0000c414       ___acrt_uninitialize       0040d414 f   MSVCRT:ucrt_stubs.obj
 0001:0000c414       ___acrt_initialize         0040d414 f   MSVCRT:ucrt_stubs.obj
 0001:0000c414       ___vcrt_uninitialize       0040d414 f   MSVCRT:ucrt_stubs.obj
 0001:0000c414       ___vcrt_initialize         0040d414 f   MSVCRT:ucrt_stubs.obj
 0001:0000c414       ___scrt_stub_for_acrt_uninitialize 0040d414 f   MSVCRT:ucrt_stubs.obj
 0001:0000c414       ___scrt_stub_for_acrt_initialize 0040d414 f   MSVCRT:ucrt_stubs.obj
 0001:0000c417       __initialize_default_precision 0040d417 f   MSVCRT:default_precision.obj
 0001:0000c438       ___local_stdio_scanf_options 0040d438 f i MSVCRT:default_local_stdio_options.obj
 0001:0000c43e       ___scrt_initialize_default_local_stdio_options 0040d43e f   MSVCRT:default_local_stdio_options.obj
 0001:0000c45b       ___scrt_is_user_matherr_present 0040d45b f   MSVCRT:matherr_detection.obj
 0001:0000c467       ___scrt_get_dyn_tls_init_callback 0040d467 f   MSVCRT:dyn_tls_init.obj
 0001:0000c46d       ___scrt_get_dyn_tls_dtor_callback 0040d46d f   MSVCRT:dyn_tls_dtor.obj
 0001:0000c473       __RTC_Initialize           0040d473 f   MSVCRT:initsect.obj
 0001:0000c49f       __RTC_Terminate            0040d49f f   MSVCRT:initsect.obj
 0001:0000c4cb       ?_Xlength_error@std@@YAXPBD@Z 0040d4cb f   msvcprt:MSVCP140.dll
 0001:0000c4d1       _IsProcessorFeaturePresent@4 0040d4d1 f   kernel32:KERNEL32.dll
 0001:0000c4d7       _memcpy                    0040d4d7 f   vcruntime:VCRUNTIME140.dll
 0001:0000c4dd       _memset                    0040d4dd f   vcruntime:VCRUNTIME140.dll
 0001:0000c4e3       _memmove                   0040d4e3 f   vcruntime:VCRUNTIME140.dll
 0001:0000c4e9       ___std_exception_copy      0040d4e9 f   vcruntime:VCRUNTIME140.dll
 0001:0000c4ef       ___std_exception_destroy   0040d4ef f   vcruntime:VCRUNTIME140.dll
 0001:0000c4f5       __CxxThrowException@8      0040d4f5 f   vcruntime:VCRUNTIME140.dll
 0001:0000c4fb       ___CxxFrameHandler3        0040d4fb f   vcruntime:VCRUNTIME140.dll
 0001:0000c501       ___current_exception       0040d501 f   vcruntime:VCRUNTIME140.dll
 0001:0000c507       ___current_exception_context 0040d507 f   vcruntime:VCRUNTIME140.dll
 0001:0000c50d       __except_handler4_common   0040d50d f   vcruntime:VCRUNTIME140.dll
 0001:0000c513       _strlen                    0040d513 f   ucrt:api-ms-win-crt-string-l1-1-0.dll
 0001:0000c519       _strcpy                    0040d519 f   ucrt:api-ms-win-crt-string-l1-1-0.dll
 0001:0000c51f       __callnewh                 0040d51f f   ucrt:api-ms-win-crt-heap-l1-1-0.dll
 0001:0000c525       _malloc                    0040d525 f   ucrt:api-ms-win-crt-heap-l1-1-0.dll
 0001:0000c52b       __configure_narrow_argv    0040d52b f   ucrt:api-ms-win-crt-runtime-l1-1-0.dll
 0001:0000c531       __initialize_narrow_environment 0040d531 f   ucrt:api-ms-win-crt-runtime-l1-1-0.dll
 0001:0000c537       __initialize_onexit_table  0040d537 f   ucrt:api-ms-win-crt-runtime-l1-1-0.dll
 0001:0000c53d       __register_onexit_function 0040d53d f   ucrt:api-ms-win-crt-runtime-l1-1-0.dll
 0001:0000c543       __crt_atexit               0040d543 f   ucrt:api-ms-win-crt-runtime-l1-1-0.dll
 0001:0000c549       __cexit                    0040d549 f   ucrt:api-ms-win-crt-runtime-l1-1-0.dll
 0001:0000c54f       __seh_filter_exe           0040d54f f   ucrt:api-ms-win-crt-runtime-l1-1-0.dll
 0001:0000c555       __set_app_type             0040d555 f   ucrt:api-ms-win-crt-runtime-l1-1-0.dll
 0001:0000c55b       ___setusermatherr          0040d55b f   ucrt:api-ms-win-crt-math-l1-1-0.dll
 0001:0000c561       __get_narrow_winmain_command_line 0040d561 f   ucrt:api-ms-win-crt-runtime-l1-1-0.dll
 0001:0000c567       __initterm                 0040d567 f   ucrt:api-ms-win-crt-runtime-l1-1-0.dll
 0001:0000c56d       __initterm_e               0040d56d f   ucrt:api-ms-win-crt-runtime-l1-1-0.dll
 0001:0000c573       _exit                      0040d573 f   ucrt:api-ms-win-crt-runtime-l1-1-0.dll
 0001:0000c579       __exit                     0040d579 f   ucrt:api-ms-win-crt-runtime-l1-1-0.dll
 0001:0000c57f       __set_fmode                0040d57f f   ucrt:api-ms-win-crt-stdio-l1-1-0.dll
 0001:0000c585       __c_exit                   0040d585 f   ucrt:api-ms-win-crt-runtime-l1-1-0.dll
 0001:0000c58b       __register_thread_local_exe_atexit_callback 0040d58b f   ucrt:api-ms-win-crt-runtime-l1-1-0.dll
 0001:0000c591       __configthreadlocale       0040d591 f   ucrt:api-ms-win-crt-locale-l1-1-0.dll
 0001:0000c597       __set_new_mode             0040d597 f   ucrt:api-ms-win-crt-heap-l1-1-0.dll
 0001:0000c59d       ___p__commode              0040d59d f   ucrt:api-ms-win-crt-stdio-l1-1-0.dll
 0001:0000c5a3       _free                      0040d5a3 f   ucrt:api-ms-win-crt-heap-l1-1-0.dll
 0001:0000c5a9       _terminate                 0040d5a9 f   ucrt:api-ms-win-crt-runtime-l1-1-0.dll
 0001:0000c5af       __controlfp_s              0040d5af f   ucrt:api-ms-win-crt-runtime-l1-1-0.dll
 0001:0000c5b5       __filter_x86_sse2_floating_point_exception_default 0040d5b5 f   MSVCRT:x86_exception_filter.obj
 0001:0000c5b5       __filter_x86_sse2_floating_point_exception 0040d5b5 f   MSVCRT:x86_exception_filter.obj
 0002:00000000       __imp__RegCreateKeyExA@36  0040e000     advapi32:ADVAPI32.dll
 0002:00000004       __imp__RegFlushKey@4       0040e004     advapi32:ADVAPI32.dll
 0002:00000008       __imp__RegOpenKeyExA@20    0040e008     advapi32:ADVAPI32.dll
 0002:0000000c       __imp__RegQueryValueExA@24 0040e00c     advapi32:ADVAPI32.dll
 0002:00000010       __imp__RegSetValueExA@24   0040e010     advapi32:ADVAPI32.dll
 0002:00000014       __imp__RegCloseKey@4       0040e014     advapi32:ADVAPI32.dll
 0002:00000018       \177ADVAPI32_NULL_THUNK_DATA 0040e018     advapi32:ADVAPI32.dll
 0002:0000001c       __imp__InitializeSListHead@4 0040e01c     kernel32:KERNEL32.dll
 0002:00000020       __imp__GetCurrentProcessId@0 0040e020     kernel32:KERNEL32.dll
 0002:00000024       __imp__QueryPerformanceCounter@4 0040e024     kernel32:KERNEL32.dll
 0002:00000028       __imp__GetStartupInfoW@4   0040e028     kernel32:KERNEL32.dll
 0002:0000002c       __imp__IsDebuggerPresent@0 0040e02c     kernel32:KERNEL32.dll
 0002:00000030       __imp__GetModuleHandleW@4  0040e030     kernel32:KERNEL32.dll
 0002:00000034       __imp__CreateEventW@16     0040e034     kernel32:KERNEL32.dll
 0002:00000038       __imp__WaitForSingleObjectEx@12 0040e038     kernel32:KERNEL32.dll
 0002:0000003c       __imp__ResetEvent@4        0040e03c     kernel32:KERNEL32.dll
 0002:00000040       __imp__SetEvent@4          0040e040     kernel32:KERNEL32.dll
 0002:00000044       __imp__DeleteCriticalSection@4 0040e044     kernel32:KERNEL32.dll
 0002:00000048       __imp__InitializeCriticalSectionAndSpinCount@8 0040e048     kernel32:KERNEL32.dll
 0002:0000004c       __imp__LeaveCriticalSection@4 0040e04c     kernel32:KERNEL32.dll
 0002:00000050       __imp__EnterCriticalSection@4 0040e050     kernel32:KERNEL32.dll
 0002:00000054       __imp__CloseHandle@4       0040e054     kernel32:KERNEL32.dll
 0002:00000058       __imp__IsProcessorFeaturePresent@4 0040e058     kernel32:KERNEL32.dll
 0002:0000005c       __imp__TerminateProcess@8  0040e05c     kernel32:KERNEL32.dll
 0002:00000060       __imp__GetCurrentProcess@0 0040e060     kernel32:KERNEL32.dll
 0002:00000064       __imp__SetUnhandledExceptionFilter@4 0040e064     kernel32:KERNEL32.dll
 0002:00000068       __imp__UnhandledExceptionFilter@4 0040e068     kernel32:KERNEL32.dll
 0002:0000006c       __imp__GetCurrentThreadId@0 0040e06c     kernel32:KERNEL32.dll
 0002:00000070       __imp__FormatMessageA@28   0040e070     kernel32:KERNEL32.dll
 0002:00000074       __imp__LocalFree@4         0040e074     kernel32:KERNEL32.dll
 0002:00000078       __imp__GetSystemTimeAsFileTime@4 0040e078     kernel32:KERNEL32.dll
 0002:0000007c       __imp__LoadLibraryA@4      0040e07c     kernel32:KERNEL32.dll
 0002:00000080       __imp__GetProcAddress@8    0040e080     kernel32:KERNEL32.dll
 0002:00000084       __imp__FreeLibrary@4       0040e084     kernel32:KERNEL32.dll
 0002:00000088       __imp__GetLastError@0      0040e088     kernel32:KERNEL32.dll
 0002:0000008c       \177KERNEL32_NULL_THUNK_DATA 0040e08c     kernel32:KERNEL32.dll
 0002:00000090       __imp_?_Xlength_error@std@@YAXPBD@Z 0040e090     msvcprt:MSVCP140.dll
 0002:00000094       \177MSVCP140_NULL_THUNK_DATA 0040e094     msvcprt:MSVCP140.dll
 0002:00000098       __imp__OffsetRect@12       0040e098     user32:USER32.dll
 0002:0000009c       __imp__GetDesktopWindow@0  0040e09c     user32:USER32.dll
 0002:000000a0       __imp__GetParent@4         0040e0a0     user32:USER32.dll
 0002:000000a4       __imp__GetTopWindow@4      0040e0a4     user32:USER32.dll
 0002:000000a8       __imp__CopyRect@8          0040e0a8     user32:USER32.dll
 0002:000000ac       __imp__SetWindowsHookExA@16 0040e0ac     user32:USER32.dll
 0002:000000b0       __imp__UnhookWindowsHookEx@4 0040e0b0     user32:USER32.dll
 0002:000000b4       __imp__CallNextHookEx@16   0040e0b4     user32:USER32.dll
 0002:000000b8       __imp__IsDialogMessageA@8  0040e0b8     user32:USER32.dll
 0002:000000bc       __imp__RegisterWindowMessageA@4 0040e0bc     user32:USER32.dll
 0002:000000c0       __imp__WindowFromPoint@8   0040e0c0     user32:USER32.dll
 0002:000000c4       __imp__GetWindow@8         0040e0c4     user32:USER32.dll
 0002:000000c8       __imp__GetWindowRect@8     0040e0c8     user32:USER32.dll
 0002:000000cc       __imp__SetWindowTextA@8    0040e0cc     user32:USER32.dll
 0002:000000d0       __imp__UpdateWindow@4      0040e0d0     user32:USER32.dll
 0002:000000d4       __imp__CheckMenuItem@12    0040e0d4     user32:USER32.dll
 0002:000000d8       __imp__GetMenu@4           0040e0d8     user32:USER32.dll
 0002:000000dc       __imp__GetSystemMetrics@4  0040e0dc     user32:USER32.dll
 0002:000000e0       __imp__TranslateAcceleratorA@12 0040e0e0     user32:USER32.dll
 0002:000000e4       __imp__LoadAcceleratorsA@8 0040e0e4     user32:USER32.dll
 0002:000000e8       __imp__EnableWindow@8      0040e0e8     user32:USER32.dll
 0002:000000ec       __imp__KillTimer@8         0040e0ec     user32:USER32.dll
 0002:000000f0       __imp__SetTimer@16         0040e0f0     user32:USER32.dll
 0002:000000f4       __imp__GetFocus@0          0040e0f4     user32:USER32.dll
 0002:000000f8       __imp__SetFocus@4          0040e0f8     user32:USER32.dll
 0002:000000fc       __imp__GetDlgCtrlID@4      0040e0fc     user32:USER32.dll
 0002:00000100       __imp__GetDlgItemInt@16    0040e100     user32:USER32.dll
 0002:00000104       __imp__GetDlgItem@8        0040e104     user32:USER32.dll
 0002:00000108       __imp__EndDialog@8         0040e108     user32:USER32.dll
 0002:0000010c       __imp__CreateDialogParamA@20 0040e10c     user32:USER32.dll
 0002:00000110       __imp__SetWindowPos@28     0040e110     user32:USER32.dll
 0002:00000114       __imp__ShowWindow@8        0040e114     user32:USER32.dll
 0002:00000118       __imp__PostQuitMessage@4   0040e118     user32:USER32.dll
 0002:0000011c       __imp__PostMessageA@16     0040e11c     user32:USER32.dll
 0002:00000120       __imp__DispatchMessageA@4  0040e120     user32:USER32.dll
 0002:00000124       __imp__TranslateMessage@4  0040e124     user32:USER32.dll
 0002:00000128       __imp__GetMessageA@16      0040e128     user32:USER32.dll
 0002:0000012c       __imp__wsprintfA           0040e12c     user32:USER32.dll
 0002:00000130       __imp__SetDlgItemTextA@12  0040e130     user32:USER32.dll
 0002:00000134       __imp__GetCursorPos@4      0040e134     user32:USER32.dll
 0002:00000138       \177USER32_NULL_THUNK_DATA 0040e138     user32:USER32.dll
 0002:0000013c       __imp__memcpy              0040e13c     vcruntime:VCRUNTIME140.dll
 0002:00000140       __imp__memset              0040e140     vcruntime:VCRUNTIME140.dll
 0002:00000144       __imp__memmove             0040e144     vcruntime:VCRUNTIME140.dll
 0002:00000148       __imp____std_exception_copy 0040e148     vcruntime:VCRUNTIME140.dll
 0002:0000014c       __imp____std_exception_destroy 0040e14c     vcruntime:VCRUNTIME140.dll
 0002:00000150       __imp___CxxThrowException@8 0040e150     vcruntime:VCRUNTIME140.dll
 0002:00000154       __imp____CxxFrameHandler3  0040e154     vcruntime:VCRUNTIME140.dll
 0002:00000158       __imp____current_exception 0040e158     vcruntime:VCRUNTIME140.dll
 0002:0000015c       __imp____current_exception_context 0040e15c     vcruntime:VCRUNTIME140.dll
 0002:00000160       __imp___except_handler4_common 0040e160     vcruntime:VCRUNTIME140.dll
 0002:00000164       \177VCRUNTIME140_NULL_THUNK_DATA 0040e164     vcruntime:VCRUNTIME140.dll
 0002:00000168       __imp__getenv              0040e168     ucrt:api-ms-win-crt-environment-l1-1-0.dll
 0002:0000016c       \177api-ms-win-crt-environment-l1-1-0_NULL_THUNK_DATA 0040e16c     ucrt:api-ms-win-crt-environment-l1-1-0.dll
 0002:00000170       __imp___set_new_mode       0040e170     ucrt:api-ms-win-crt-heap-l1-1-0.dll
 0002:00000174       __imp__malloc              0040e174     ucrt:api-ms-win-crt-heap-l1-1-0.dll
 0002:00000178       __imp___callnewh           0040e178     ucrt:api-ms-win-crt-heap-l1-1-0.dll
 0002:0000017c       __imp__free                0040e17c     ucrt:api-ms-win-crt-heap-l1-1-0.dll
 0002:00000180       \177api-ms-win-crt-heap-l1-1-0_NULL_THUNK_DATA 0040e180     ucrt:api-ms-win-crt-heap-l1-1-0.dll
 0002:00000184       __imp___configthreadlocale 0040e184     ucrt:api-ms-win-crt-locale-l1-1-0.dll
 0002:00000188       \177api-ms-win-crt-locale-l1-1-0_NULL_THUNK_DATA 0040e188     ucrt:api-ms-win-crt-locale-l1-1-0.dll
 0002:0000018c       __imp____setusermatherr    0040e18c     ucrt:api-ms-win-crt-math-l1-1-0.dll
 0002:00000190       \177api-ms-win-crt-math-l1-1-0_NULL_THUNK_DATA 0040e190     ucrt:api-ms-win-crt-math-l1-1-0.dll
 0002:00000194       __imp___controlfp_s        0040e194     ucrt:api-ms-win-crt-runtime-l1-1-0.dll
 0002:00000198       __imp__terminate           0040e198     ucrt:api-ms-win-crt-runtime-l1-1-0.dll
 0002:0000019c       __imp___register_thread_local_exe_atexit_callback 0040e19c     ucrt:api-ms-win-crt-runtime-l1-1-0.dll
 0002:000001a0       __imp___c_exit             0040e1a0     ucrt:api-ms-win-crt-runtime-l1-1-0.dll
 0002:000001a4       __imp___invalid_parameter_noinfo_noreturn 0040e1a4     ucrt:api-ms-win-crt-runtime-l1-1-0.dll
 0002:000001a8       __imp___exit               0040e1a8     ucrt:api-ms-win-crt-runtime-l1-1-0.dll
 0002:000001ac       __imp__exit                0040e1ac     ucrt:api-ms-win-crt-runtime-l1-1-0.dll
 0002:000001b0       __imp___configure_narrow_argv 0040e1b0     ucrt:api-ms-win-crt-runtime-l1-1-0.dll
 0002:000001b4       __imp___initialize_narrow_environment 0040e1b4     ucrt:api-ms-win-crt-runtime-l1-1-0.dll
 0002:000001b8       __imp___initialize_onexit_table 0040e1b8     ucrt:api-ms-win-crt-runtime-l1-1-0.dll
 0002:000001bc       __imp___register_onexit_function 0040e1bc     ucrt:api-ms-win-crt-runtime-l1-1-0.dll
 0002:000001c0       __imp___crt_atexit         0040e1c0     ucrt:api-ms-win-crt-runtime-l1-1-0.dll
 0002:000001c4       __imp___initterm_e         0040e1c4     ucrt:api-ms-win-crt-runtime-l1-1-0.dll
 0002:000001c8       __imp___cexit              0040e1c8     ucrt:api-ms-win-crt-runtime-l1-1-0.dll
 0002:000001cc       __imp___seh_filter_exe     0040e1cc     ucrt:api-ms-win-crt-runtime-l1-1-0.dll
 0002:000001d0       __imp___set_app_type       0040e1d0     ucrt:api-ms-win-crt-runtime-l1-1-0.dll
 0002:000001d4       __imp___get_narrow_winmain_command_line 0040e1d4     ucrt:api-ms-win-crt-runtime-l1-1-0.dll
 0002:000001d8       __imp___initterm           0040e1d8     ucrt:api-ms-win-crt-runtime-l1-1-0.dll
 0002:000001dc       \177api-ms-win-crt-runtime-l1-1-0_NULL_THUNK_DATA 0040e1dc     ucrt:api-ms-win-crt-runtime-l1-1-0.dll
 0002:000001e0       __imp____stdio_common_vfprintf 0040e1e0     ucrt:api-ms-win-crt-stdio-l1-1-0.dll
 0002:000001e4       __imp___set_fmode          0040e1e4     ucrt:api-ms-win-crt-stdio-l1-1-0.dll
 0002:000001e8       __imp__fflush              0040e1e8     ucrt:api-ms-win-crt-stdio-l1-1-0.dll
 0002:000001ec       __imp__fopen               0040e1ec     ucrt:api-ms-win-crt-stdio-l1-1-0.dll
 0002:000001f0       __imp__fclose              0040e1f0     ucrt:api-ms-win-crt-stdio-l1-1-0.dll
 0002:000001f4       __imp____stdio_common_vfwprintf 0040e1f4     ucrt:api-ms-win-crt-stdio-l1-1-0.dll
 0002:000001f8       __imp____acrt_iob_func     0040e1f8     ucrt:api-ms-win-crt-stdio-l1-1-0.dll
 0002:000001fc       __imp____p__commode        0040e1fc     ucrt:api-ms-win-crt-stdio-l1-1-0.dll
 0002:00000200       __imp____stdio_common_vsprintf 0040e200     ucrt:api-ms-win-crt-stdio-l1-1-0.dll
 0002:00000204       \177api-ms-win-crt-stdio-l1-1-0_NULL_THUNK_DATA 0040e204     ucrt:api-ms-win-crt-stdio-l1-1-0.dll
 0002:00000208       __imp__strlen              0040e208     ucrt:api-ms-win-crt-string-l1-1-0.dll
 0002:0000020c       __imp__strncpy             0040e20c     ucrt:api-ms-win-crt-string-l1-1-0.dll
 0002:00000210       __imp__strcpy              0040e210     ucrt:api-ms-win-crt-string-l1-1-0.dll
 0002:00000214       __imp__strncat             0040e214     ucrt:api-ms-win-crt-string-l1-1-0.dll
 0002:00000218       \177api-ms-win-crt-string-l1-1-0_NULL_THUNK_DATA 0040e218     ucrt:api-ms-win-crt-string-l1-1-0.dll
 0002:0000021c       __imp___localtime64        0040e21c     ucrt:api-ms-win-crt-time-l1-1-0.dll
 0002:00000220       __imp___time64             0040e220     ucrt:api-ms-win-crt-time-l1-1-0.dll
 0002:00000224       __imp__asctime             0040e224     ucrt:api-ms-win-crt-time-l1-1-0.dll
 0002:00000228       \177api-ms-win-crt-time-l1-1-0_NULL_THUNK_DATA 0040e228     ucrt:api-ms-win-crt-time-l1-1-0.dll
 0002:0000022c       ___guard_check_icall_fptr  0040e22c     MSVCRT:guard_support.obj
 0002:00000230       ___xc_a                    0040e230     MSVCRT:initializers.obj
 0002:0000023c       ___xc_z                    0040e23c     MSVCRT:initializers.obj
 0002:00000240       ___xi_a                    0040e240     MSVCRT:initializers.obj
 0002:00000250       ___xi_z                    0040e250     MSVCRT:initializers.obj
 0002:00000254       ___xl_a                    0040e254     MSVCRT:tlssup.obj
 0002:00000258       ___xl_z                    0040e258     MSVCRT:tlssup.obj
 0002:0000025c       ___xp_a                    0040e25c     MSVCRT:initializers.obj
 0002:00000260       ___xp_z                    0040e260     MSVCRT:initializers.obj
 0002:00000264       ___xt_a                    0040e264     MSVCRT:initializers.obj
 0002:00000268       ___xt_z                    0040e268     MSVCRT:initializers.obj
 0002:00001958       ??_7exception@std@@6B@     0040f958     MessageHistory.obj
 0002:00001960       ??_C@_0BC@EOODALEL@Unknown?5exception@ 0040f960     MessageHistory.obj
 0002:00001978       ??_7bad_alloc@std@@6B@     0040f978     MessageHistory.obj
 0002:00001984       ??_7bad_array_new_length@std@@6B@ 0040f984     MessageHistory.obj
 0002:0000198c       ??_C@_0BF@KINCDENJ@bad?5array?5new?5length@ 0040f98c     MessageHistory.obj
 0002:000019a4       ??_C@_0BA@JFNIOLAK@string?5too?5long@ 0040f9a4     MessageHistory.obj
 0002:000019b4       ??_C@_0O@NKNMEGII@list?5too?5long@ 0040f9b4     MessageHistory.obj
 0002:000021a4       ??_7type_info@@6B@         004101a4     MSVCRT:std_type_info_static.obj
 0002:000021a8       ??_C@_1EC@JIJBPKFM@?$AAa?$AAp?$AAi?$AA?9?$AAm?$AAs?$AA?9?$AAw?$AAi?$AAn?$AA?9?$AAc?$AAo?$AAr?$AAe@ 004101a8     MSVCRT:thread_safe_statics.obj
 0002:000021ec       ??_C@_1BK@MGMFAEKH@?$AAk?$AAe?$AAr?$AAn?$AAe?$AAl?$AA3?$AA2?$AA?4?$AAd?$AAl?$AAl@ 004101ec     MSVCRT:thread_safe_statics.obj
 0002:00002208       ??_C@_0BJ@JEBJOJFJ@SleepConditionVariableCS@ 00410208     MSVCRT:thread_safe_statics.obj
 0002:00002224       ??_C@_0BJ@PGPPEPCC@WakeAllConditionVariable@ 00410224     MSVCRT:thread_safe_statics.obj
 0002:00002240       ??_C@_0P@GHFPNOJB@bad?5allocation@ 00410240     MSVCRT:throw_bad_alloc.obj
 0002:000022c0       __load_config_used         004102c0     MSVCRT:loadcfg.obj
 0002:00002378       __tls_used                 00410378     MSVCRT:tlssup.obj
 0002:00002390       ??_R4exception@std@@6B@    00410390     MessageHistory.obj
 0002:000023a4       ??_R3exception@std@@8      004103a4     MessageHistory.obj
 0002:000023b4       ??_R2exception@std@@8      004103b4     MessageHistory.obj
 0002:000023bc       ??_R1A@?0A@EA@exception@std@@8 004103bc     MessageHistory.obj
 0002:000023d8       ??_R4bad_alloc@std@@6B@    004103d8     MessageHistory.obj
 0002:000023ec       ??_R3bad_alloc@std@@8      004103ec     MessageHistory.obj
 0002:000023fc       ??_R2bad_alloc@std@@8      004103fc     MessageHistory.obj
 0002:00002408       ??_R1A@?0A@EA@bad_alloc@std@@8 00410408     MessageHistory.obj
 0002:00002424       ??_R4bad_array_new_length@std@@6B@ 00410424     MessageHistory.obj
 0002:00002438       ??_R3bad_array_new_length@std@@8 00410438     MessageHistory.obj
 0002:00002448       ??_R2bad_array_new_length@std@@8 00410448     MessageHistory.obj
 0002:00002458       ??_R1A@?0A@EA@bad_array_new_length@std@@8 00410458     MessageHistory.obj
 0002:00002474       ??_R4type_info@@6B@        00410474     MSVCRT:std_type_info_static.obj
 0002:00002488       ??_R3type_info@@8          00410488     MSVCRT:std_type_info_static.obj
 0002:00002498       ??_R2type_info@@8          00410498     MSVCRT:std_type_info_static.obj
 0002:000024a0       ??_R1A@?0A@EA@type_info@@8 004104a0     MSVCRT:std_type_info_static.obj
 0002:000024bc       ___safe_se_handler_table   004104bc     <linker-defined>
 0002:0000288c       ___rtc_iaa                 0041088c     MSVCRT:initsect.obj
 0002:00002890       ___rtc_izz                 00410890     MSVCRT:initsect.obj
 0002:00002894       ___rtc_taa                 00410894     MSVCRT:initsect.obj
 0002:00002898       ___rtc_tzz                 00410898     MSVCRT:initsect.obj
 0002:0000289c       __tls_start                0041089c     MSVCRT:tlssup.obj
 0002:000028a0       __Init_thread_epoch        004108a0     MSVCRT:thread_safe_statics.obj
 0002:000028a4       __tls_end                  004108a4     MSVCRT:tlssup.obj
 0002:00002950       __TI3?AVbad_array_new_length@std@@ 00410950     MessageHistory.obj
 0002:00002960       __CTA3?AVbad_array_new_length@std@@ 00410960     MessageHistory.obj
 0002:00002970       __CT??_R0?AVbad_array_new_length@std@@@8??0bad_array_new_length@std@@QAE@ABV01@@Z12 00410970     MessageHistory.obj
 0002:0000298c       __CT??_R0?AVbad_alloc@std@@@8??0bad_alloc@std@@QAE@ABV01@@Z12 0041098c     MessageHistory.obj
 0002:000029a8       __CT??_R0?AVexception@std@@@8??0exception@std@@QAE@ABV01@@Z12 004109a8     MessageHistory.obj
 0002:00002a04       __TI2?AVbad_alloc@std@@    00410a04     MSVCRT:throw_bad_alloc.obj
 0002:00002a14       __CTA2?AVbad_alloc@std@@   00410a14     MSVCRT:throw_bad_alloc.obj
 0002:00002a20       __IMPORT_DESCRIPTOR_ADVAPI32 00410a20     advapi32:ADVAPI32.dll
 0002:00002a34       __IMPORT_DESCRIPTOR_USER32 00410a34     user32:USER32.dll
 0002:00002a48       __IMPORT_DESCRIPTOR_MSVCP140 00410a48     msvcprt:MSVCP140.dll
 0002:00002a5c       __IMPORT_DESCRIPTOR_KERNEL32 00410a5c     kernel32:KERNEL32.dll
 0002:00002a70       __IMPORT_DESCRIPTOR_VCRUNTIME140 00410a70     vcruntime:VCRUNTIME140.dll
 0002:00002a84       __IMPORT_DESCRIPTOR_api-ms-win-crt-string-l1-1-0 00410a84     ucrt:api-ms-win-crt-string-l1-1-0.dll
 0002:00002a98       __IMPORT_DESCRIPTOR_api-ms-win-crt-stdio-l1-1-0 00410a98     ucrt:api-ms-win-crt-stdio-l1-1-0.dll
 0002:00002aac       __IMPORT_DESCRIPTOR_api-ms-win-crt-environment-l1-1-0 00410aac     ucrt:api-ms-win-crt-environment-l1-1-0.dll
 0002:00002ac0       __IMPORT_DESCRIPTOR_api-ms-win-crt-time-l1-1-0 00410ac0     ucrt:api-ms-win-crt-time-l1-1-0.dll
 0002:00002ad4       __IMPORT_DESCRIPTOR_api-ms-win-crt-runtime-l1-1-0 00410ad4     ucrt:api-ms-win-crt-runtime-l1-1-0.dll
 0002:00002ae8       __IMPORT_DESCRIPTOR_api-ms-win-crt-heap-l1-1-0 00410ae8     ucrt:api-ms-win-crt-heap-l1-1-0.dll
 0002:00002afc       __IMPORT_DESCRIPTOR_api-ms-win-crt-math-l1-1-0 00410afc     ucrt:api-ms-win-crt-math-l1-1-0.dll
 0002:00002b10       __IMPORT_DESCRIPTOR_api-ms-win-crt-locale-l1-1-0 00410b10     ucrt:api-ms-win-crt-locale-l1-1-0.dll
 0002:00002b24       __NULL_IMPORT_DESCRIPTOR   00410b24     advapi32:ADVAPI32.dll
 0003:00000a64       ?sm_MaxMessages@MessageHistory@@2IA 00412a64     MessageHistory.obj
 0003:00000a68       ?szAppName@@3PADA          00412a68     jaccessinspector.obj
 0003:00000a80       ___security_cookie_complement 00412a80     MSVCRT:gs_cookie.obj
 0003:00000a84       ___security_cookie         00412a84     MSVCRT:gs_cookie.obj
 0003:00000a88       __fltused                  00412a88     MSVCRT:fltused.obj
 0003:00000a8c       ___scrt_native_dllmain_reason 00412a8c     MSVCRT:utility.obj
 0003:00000a90       __Init_global_epoch        00412a90     MSVCRT:thread_safe_statics.obj
 0003:00000a94       ___isa_enabled             00412a94     MSVCRT:cpu_disp.obj
 0003:00000aa0       ___scrt_default_matherr    00412aa0     MSVCRT:matherr.obj
 0003:00000aa4       ___scrt_ucrt_dll_is_in_use 00412aa4     MSVCRT:ucrt_stubs.obj
 0003:00000aa8       ??_R0?AVbad_array_new_length@std@@@8 00412aa8     MessageHistory.obj
 0003:00000ad0       ??_R0?AVbad_alloc@std@@@8  00412ad0     MessageHistory.obj
 0003:00000aec       ??_R0?AVexception@std@@@8  00412aec     MessageHistory.obj
 0003:00000b08       ??_R0?AVtype_info@@@8      00412b08     MSVCRT:std_type_info_static.obj
 0003:00000b20       _theAccessBridgeInitializedFlag 00412b20     AccessBridgeCalls.obj
 0003:00000b28       ?_OptionsStorage@?1??__local_stdio_printf_options@@9@4_KA 00412b28     AccessBridgeDebug.obj
 0003:00000c38       ?theFromJavaHelloMsgID@@3IA 00412c38     AccessBridgeMessages.obj
 0003:00000c3c       ?theFromWindowsHelloMsgID@@3IA 00412c3c     AccessBridgeMessages.obj
 0003:00000c40       ?g_LogStringCallback@@3P6GXPBD@ZA 00412c40     AccessInfo.obj
 0003:00000c88       ?theDialogWindow@@3PAUHWND__@@A 00412c88     jaccessinspector.obj
 0003:00000c8c       ?theGoToDialogWindow@@3PAUHWND__@@A 00412c8c     jaccessinspector.obj
 0003:00000c90       ?theInstance@@3PAUHINSTANCE__@@A 00412c90     jaccessinspector.obj
 0003:00000c94       ?theAccessBridgeLoadedFlag@@3HA 00412c94     jaccessinspector.obj
 0003:00000c98       ?prevKbdHook@@3PAUHHOOK__@@A 00412c98     jaccessinspector.obj
 0003:00000c9c       ?prevMouseHook@@3PAUHHOOK__@@A 00412c9c     jaccessinspector.obj
 0003:00000ca0       ?updateMouse@@3HA          00412ca0     jaccessinspector.obj
 0003:00000ca4       ?updateF1@@3HA             00412ca4     jaccessinspector.obj
 0003:00000ca8       ?updateF2@@3HA             00412ca8     jaccessinspector.obj
 0003:00000cac       ?trackMouse@@3HA           00412cac     jaccessinspector.obj
 0003:00000cb0       ?trackMouseExited@@3HA     00412cb0     jaccessinspector.obj
 0003:00000cb4       ?trackMouseClicked@@3HA    00412cb4     jaccessinspector.obj
 0003:00000cb8       ?trackMousePressed@@3HA    00412cb8     jaccessinspector.obj
 0003:00000cbc       ?trackMouseReleased@@3HA   00412cbc     jaccessinspector.obj
 0003:00000cc0       ?trackFocus@@3HA           00412cc0     jaccessinspector.obj
 0003:00000cc4       ?trackFocusLost@@3HA       00412cc4     jaccessinspector.obj
 0003:00000cc8       ?trackCaret@@3HA           00412cc8     jaccessinspector.obj
 0003:00000ccc       ?trackShutdown@@3HA        00412ccc     jaccessinspector.obj
 0003:00000cd0       ?trackMenuSelected@@3HA    00412cd0     jaccessinspector.obj
 0003:00000cd4       ?trackMenuDeselected@@3HA  00412cd4     jaccessinspector.obj
 0003:00000cd8       ?trackMenuCanceled@@3HA    00412cd8     jaccessinspector.obj
 0003:00000cdc       ?trackPopupVisible@@3HA    00412cdc     jaccessinspector.obj
 0003:00000ce0       ?trackPopupInvisible@@3HA  00412ce0     jaccessinspector.obj
 0003:00000ce4       ?trackPopupCanceled@@3HA   00412ce4     jaccessinspector.obj
 0003:00000ce8       ?trackPropertyNameChange@@3HA 00412ce8     jaccessinspector.obj
 0003:00000cec       ?trackPropertyDescriptionChange@@3HA 00412cec     jaccessinspector.obj
 0003:00000cf0       ?trackPropertyStateChange@@3HA 00412cf0     jaccessinspector.obj
 0003:00000cf4       ?trackPropertyValueChange@@3HA 00412cf4     jaccessinspector.obj
 0003:00000cf8       ?trackPropertySelectionChange@@3HA 00412cf8     jaccessinspector.obj
 0003:00000cfc       ?trackPropertyTextChange@@3HA 00412cfc     jaccessinspector.obj
 0003:00000d00       ?trackPropertyCaretChange@@3HA 00412d00     jaccessinspector.obj
 0003:00000d04       ?trackPropertyVisibleDataChange@@3HA 00412d04     jaccessinspector.obj
 0003:00000d08       ?trackPropertyChildChange@@3HA 00412d08     jaccessinspector.obj
 0003:00000d0c       ?trackPropertyActiveDescendentChange@@3HA 00412d0c     jaccessinspector.obj
 0003:00000d10       ?trackPropertyTableModelChange@@3HA 00412d10     jaccessinspector.obj
 0003:00000d14       ?logfile@@3PAU_iobuf@@A    00412d14     jaccessinspector.obj
 0003:00000d18       ?g_MessageHistory@@3VMessageHistory@@A 00412d18     jaccessinspector.obj
 0003:0000106c       ___scrt_current_native_startup_state 0041306c     MSVCRT:utility.obj
 0003:00001070       ___scrt_native_startup_lock 00413070     MSVCRT:utility.obj
 0003:000010b8       __tls_index                004130b8     MSVCRT:tlssup.obj
 0003:000010bc       ___isa_available           004130bc     MSVCRT:cpu_disp.obj
 0003:000010c0       ___favor                   004130c0     MSVCRT:cpu_disp.obj
 0003:000010c4       ___scrt_debugger_hook_flag 004130c4     MSVCRT:utility_desktop.obj
 0003:000010c8       ?__type_info_root_node@@3U__type_info_node@@A 004130c8     MSVCRT:tncleanup.obj
 0003:000010d0       ?_OptionsStorage@?1??__local_stdio_scanf_options@@9@4_KA 004130d0     MSVCRT:default_local_stdio_options.obj
 0003:000010e0       _theAccessBridge           004130e0     <common>
 0003:00001264       _theAccessBridgeInstance   00413264     <common>
 0003:00001268       ___dyn_tls_dtor_callback   00413268     <common>
 0003:0000126c       ___dyn_tls_init_callback   0041326c     <common>

 entry point at        0001:0000be95

 Static symbols

 0000:fffe8000       .debug$S                   00400000     msvcprt:MSVCP140.dll
 0000:fffe8000       .debug$S                   00400000     vcruntime:VCRUNTIME140.dll
 0000:fffe8000       .debug$S                   00400000     vcruntime:VCRUNTIME140.dll
 0000:fffe8000       .debug$S                   00400000     vcruntime:VCRUNTIME140.dll
 0000:fffe8000       .debug$S                   00400000     vcruntime:VCRUNTIME140.dll
 0000:fffe8000       .debug$S                   00400000     vcruntime:VCRUNTIME140.dll
 0000:fffe8000       .debug$S                   00400000     vcruntime:VCRUNTIME140.dll
 0000:fffe8000       .debug$S                   00400000     vcruntime:VCRUNTIME140.dll
 0000:fffe8000       .debug$S                   00400000     vcruntime:VCRUNTIME140.dll
 0000:fffe8000       .debug$S                   00400000     vcruntime:VCRUNTIME140.dll
 0000:fffe8000       .debug$S                   00400000     vcruntime:VCRUNTIME140.dll
 0000:fffe8000       .debug$S                   00400000     vcruntime:VCRUNTIME140.dll
 0000:fffe8000       .debug$S                   00400000     ucrt:api-ms-win-crt-environment-l1-1-0.dll
 0000:fffe8000       .debug$S                   00400000     ucrt:api-ms-win-crt-heap-l1-1-0.dll
 0000:fffe8000       .debug$S                   00400000     ucrt:api-ms-win-crt-heap-l1-1-0.dll
 0000:fffe8000       .debug$S                   00400000     ucrt:api-ms-win-crt-heap-l1-1-0.dll
 0000:fffe8000       .debug$S                   00400000     ucrt:api-ms-win-crt-heap-l1-1-0.dll
 0000:fffe8000       .debug$S                   00400000     ucrt:api-ms-win-crt-locale-l1-1-0.dll
 0000:fffe8000       .debug$S                   00400000     ucrt:api-ms-win-crt-math-l1-1-0.dll
 0000:fffe8000       .debug$S                   00400000     ucrt:api-ms-win-crt-runtime-l1-1-0.dll
 0000:fffe8000       .debug$S                   00400000     ucrt:api-ms-win-crt-runtime-l1-1-0.dll
 0000:fffe8000       .debug$S                   00400000     ucrt:api-ms-win-crt-runtime-l1-1-0.dll
 0000:fffe8000       .debug$S                   00400000     ucrt:api-ms-win-crt-runtime-l1-1-0.dll
 0000:fffe8000       .debug$S                   00400000     ucrt:api-ms-win-crt-runtime-l1-1-0.dll
 0000:fffe8000       .debug$S                   00400000     ucrt:api-ms-win-crt-runtime-l1-1-0.dll
 0000:fffe8000       .debug$S                   00400000     ucrt:api-ms-win-crt-runtime-l1-1-0.dll
 0000:fffe8000       .debug$S                   00400000     ucrt:api-ms-win-crt-runtime-l1-1-0.dll
 0000:fffe8000       .debug$S                   00400000     ucrt:api-ms-win-crt-runtime-l1-1-0.dll
 0000:fffe8000       .debug$S                   00400000     ucrt:api-ms-win-crt-runtime-l1-1-0.dll
 0000:fffe8000       .debug$S                   00400000     ucrt:api-ms-win-crt-runtime-l1-1-0.dll
 0000:fffe8000       .debug$S                   00400000     ucrt:api-ms-win-crt-runtime-l1-1-0.dll
 0000:fffe8000       .debug$S                   00400000     ucrt:api-ms-win-crt-runtime-l1-1-0.dll
 0000:fffe8000       .debug$S                   00400000     ucrt:api-ms-win-crt-runtime-l1-1-0.dll
 0000:fffe8000       .debug$S                   00400000     ucrt:api-ms-win-crt-runtime-l1-1-0.dll
 0000:fffe8000       .debug$S                   00400000     ucrt:api-ms-win-crt-runtime-l1-1-0.dll
 0000:fffe8000       .debug$S                   00400000     ucrt:api-ms-win-crt-runtime-l1-1-0.dll
 0000:fffe8000       .debug$S                   00400000     ucrt:api-ms-win-crt-runtime-l1-1-0.dll
 0000:fffe8000       .debug$S                   00400000     ucrt:api-ms-win-crt-runtime-l1-1-0.dll
 0000:fffe8000       .debug$S                   00400000     ucrt:api-ms-win-crt-runtime-l1-1-0.dll
 0000:fffe8000       .debug$S                   00400000     ucrt:api-ms-win-crt-runtime-l1-1-0.dll
 0000:fffe8000       .debug$S                   00400000     ucrt:api-ms-win-crt-stdio-l1-1-0.dll
 0000:fffe8000       .debug$S                   00400000     ucrt:api-ms-win-crt-stdio-l1-1-0.dll
 0000:fffe8000       .debug$S                   00400000     ucrt:api-ms-win-crt-stdio-l1-1-0.dll
 0000:fffe8000       .debug$S                   00400000     ucrt:api-ms-win-crt-stdio-l1-1-0.dll
 0000:fffe8000       .debug$S                   00400000     ucrt:api-ms-win-crt-stdio-l1-1-0.dll
 0000:fffe8000       .debug$S                   00400000     ucrt:api-ms-win-crt-stdio-l1-1-0.dll
 0000:fffe8000       .debug$S                   00400000     ucrt:api-ms-win-crt-stdio-l1-1-0.dll
 0000:fffe8000       .debug$S                   00400000     ucrt:api-ms-win-crt-stdio-l1-1-0.dll
 0000:fffe8000       .debug$S                   00400000     ucrt:api-ms-win-crt-stdio-l1-1-0.dll
 0000:fffe8000       .debug$S                   00400000     ucrt:api-ms-win-crt-string-l1-1-0.dll
 0000:fffe8000       .debug$S                   00400000     ucrt:api-ms-win-crt-string-l1-1-0.dll
 0000:fffe8000       .debug$S                   00400000     ucrt:api-ms-win-crt-string-l1-1-0.dll
 0000:fffe8000       .debug$S                   00400000     ucrt:api-ms-win-crt-string-l1-1-0.dll
 0000:fffe8000       .debug$S                   00400000     ucrt:api-ms-win-crt-time-l1-1-0.dll
 0000:fffe8000       .debug$S                   00400000     ucrt:api-ms-win-crt-time-l1-1-0.dll
 0000:fffe8000       .debug$S                   00400000     ucrt:api-ms-win-crt-time-l1-1-0.dll
 0000:fffe8000       .debug$S                   00400000     advapi32:ADVAPI32.dll
 0000:fffe8000       .debug$S                   00400000     advapi32:ADVAPI32.dll
 0000:fffe8000       .debug$S                   00400000     advapi32:ADVAPI32.dll
 0000:fffe8000       .debug$S                   00400000     advapi32:ADVAPI32.dll
 0000:fffe8000       .debug$S                   00400000     advapi32:ADVAPI32.dll
 0000:fffe8000       .debug$S                   00400000     advapi32:ADVAPI32.dll
 0000:fffe8000       .debug$S                   00400000     kernel32:KERNEL32.dll
 0000:fffe8000       .debug$S                   00400000     kernel32:KERNEL32.dll
 0000:fffe8000       .debug$S                   00400000     kernel32:KERNEL32.dll
 0000:fffe8000       .debug$S                   00400000     kernel32:KERNEL32.dll
 0000:fffe8000       .debug$S                   00400000     kernel32:KERNEL32.dll
 0000:fffe8000       .debug$S                   00400000     kernel32:KERNEL32.dll
 0000:fffe8000       .debug$S                   00400000     kernel32:KERNEL32.dll
 0000:fffe8000       .debug$S                   00400000     kernel32:KERNEL32.dll
 0000:fffe8000       .debug$S                   00400000     kernel32:KERNEL32.dll
 0000:fffe8000       .debug$S                   00400000     kernel32:KERNEL32.dll
 0000:fffe8000       .debug$S                   00400000     kernel32:KERNEL32.dll
 0000:fffe8000       .debug$S                   00400000     kernel32:KERNEL32.dll
 0000:fffe8000       .debug$S                   00400000     kernel32:KERNEL32.dll
 0000:fffe8000       .debug$S                   00400000     kernel32:KERNEL32.dll
 0000:fffe8000       .debug$S                   00400000     kernel32:KERNEL32.dll
 0000:fffe8000       .debug$S                   00400000     kernel32:KERNEL32.dll
 0000:fffe8000       .debug$S                   00400000     kernel32:KERNEL32.dll
 0000:fffe8000       .debug$S                   00400000     kernel32:KERNEL32.dll
 0000:fffe8000       .debug$S                   00400000     kernel32:KERNEL32.dll
 0000:fffe8000       .debug$S                   00400000     kernel32:KERNEL32.dll
 0000:fffe8000       .debug$S                   00400000     kernel32:KERNEL32.dll
 0000:fffe8000       .debug$S                   00400000     kernel32:KERNEL32.dll
 0000:fffe8000       .debug$S                   00400000     kernel32:KERNEL32.dll
 0000:fffe8000       .debug$S                   00400000     kernel32:KERNEL32.dll
 0000:fffe8000       .debug$S                   00400000     kernel32:KERNEL32.dll
 0000:fffe8000       .debug$S                   00400000     kernel32:KERNEL32.dll
 0000:fffe8000       .debug$S                   00400000     kernel32:KERNEL32.dll
 0000:fffe8000       .debug$S                   00400000     kernel32:KERNEL32.dll
 0000:fffe8000       .debug$S                   00400000     user32:USER32.dll
 0000:fffe8000       .debug$S                   00400000     user32:USER32.dll
 0000:fffe8000       .debug$S                   00400000     user32:USER32.dll
 0000:fffe8000       .debug$S                   00400000     user32:USER32.dll
 0000:fffe8000       .debug$S                   00400000     user32:USER32.dll
 0000:fffe8000       .debug$S                   00400000     user32:USER32.dll
 0000:fffe8000       .debug$S                   00400000     user32:USER32.dll
 0000:fffe8000       .debug$S                   00400000     user32:USER32.dll
 0000:fffe8000       .debug$S                   00400000     user32:USER32.dll
 0000:fffe8000       .debug$S                   00400000     user32:USER32.dll
 0000:fffe8000       .debug$S                   00400000     user32:USER32.dll
 0000:fffe8000       .debug$S                   00400000     user32:USER32.dll
 0000:fffe8000       .debug$S                   00400000     user32:USER32.dll
 0000:fffe8000       .debug$S                   00400000     user32:USER32.dll
 0000:fffe8000       .debug$S                   00400000     user32:USER32.dll
 0000:fffe8000       .debug$S                   00400000     user32:USER32.dll
 0000:fffe8000       .debug$S                   00400000     user32:USER32.dll
 0000:fffe8000       .debug$S                   00400000     user32:USER32.dll
 0000:fffe8000       .debug$S                   00400000     user32:USER32.dll
 0000:fffe8000       .debug$S                   00400000     user32:USER32.dll
 0000:fffe8000       .debug$S                   00400000     user32:USER32.dll
 0000:fffe8000       .debug$S                   00400000     user32:USER32.dll
 0000:fffe8000       .debug$S                   00400000     user32:USER32.dll
 0000:fffe8000       .debug$S                   00400000     user32:USER32.dll
 0000:fffe8000       .debug$S                   00400000     user32:USER32.dll
 0000:fffe8000       .debug$S                   00400000     user32:USER32.dll
 0000:fffe8000       .debug$S                   00400000     user32:USER32.dll
 0000:fffe8000       .debug$S                   00400000     user32:USER32.dll
 0000:fffe8000       .debug$S                   00400000     user32:USER32.dll
 0000:fffe8000       .debug$S                   00400000     user32:USER32.dll
 0000:fffe8000       .debug$S                   00400000     user32:USER32.dll
 0000:fffe8000       .debug$S                   00400000     user32:USER32.dll
 0000:fffe8000       .debug$S                   00400000     user32:USER32.dll
 0000:fffe8000       .debug$S                   00400000     user32:USER32.dll
 0000:fffe8000       .debug$S                   00400000     user32:USER32.dll
 0000:fffe8000       .debug$S                   00400000     user32:USER32.dll
 0000:fffe8000       .debug$S                   00400000     user32:USER32.dll
 0000:fffe8000       .debug$S                   00400000     user32:USER32.dll
 0000:fffe8000       .debug$S                   00400000     user32:USER32.dll
 0000:fffe8000       .debug$S                   00400000     user32:USER32.dll
 0001:00000000       ??__Eg_MessageHistory@@YAXXZ 00401000 f   jaccessinspector.obj
 0001:000047e0       _localtime                 004057e0 f   AccessInfo.obj
 0001:00004800       _time                      00405800 f   AccessInfo.obj
 0001:00008138       $LN132                     00409138     jaccessinspector.obj
 0001:0000814c       $LN131                     0040914c     jaccessinspector.obj
 0001:00008170       $LN133                     00409170     jaccessinspector.obj
 0001:00008180       $LN135                     00409180     jaccessinspector.obj
 0001:000081b8       $LN134                     004091b8     jaccessinspector.obj
 0001:00008284       $LN136                     00409284     jaccessinspector.obj
 0001:0000b710       $$000000                   0040c710     MSVCRT:ulldiv.obj
 0001:0000b790       $$000000                   0040c790     MSVCRT:chkstk.obj
 0001:0000b81e       ?find_pe_section@@YAPAU_IMAGE_SECTION_HEADER@@QAEI@Z 0040c81e f   MSVCRT:utility.obj
 0001:0000ba6f       ?__scrt_initialize_thread_safe_statics@@YAHXZ 0040ca6f f   MSVCRT:thread_safe_statics.obj
 0001:0000ba96       ?__scrt_initialize_thread_safe_statics_platform_specific@@YAXXZ 0040ca96 f   MSVCRT:thread_safe_statics.obj
 0001:0000bb18       ?__scrt_uninitialize_thread_safe_statics@@YAXXZ 0040cb18 f   MSVCRT:thread_safe_statics.obj
 0001:0000bc54       ?pre_c_initialization@@YAHXZ 0040cc54 f   MSVCRT:exe_winmain.obj
 0001:0000bcff       ?post_pgo_initialization@@YAHXZ 0040ccff f   MSVCRT:exe_winmain.obj
 0001:0000bd07       ?pre_cpp_initialization@@YAXXZ 0040cd07 f   MSVCRT:exe_winmain.obj
 0001:0000bd19       ?__scrt_common_main_seh@@YAHXZ 0040cd19 f   MSVCRT:exe_winmain.obj
 0001:0000c2e0       $$000000                   0040d2e0     MSVCRT:sehprolg4.obj
 0001:0000c36a       ___get_entropy             0040d36a f   MSVCRT:gs_support.obj
 0001:0000c630       __unwindfunclet$?AddMessage@MessageHistory@@QAEXPBD@Z$0 0040d630 f   MessageHistory.obj
 0001:0000c63d       __ehhandler$?AddMessage@MessageHistory@@QAEXPBD@Z 0040d63d f   MessageHistory.obj
 0001:0000c670       __unwindfunclet$??$?0V?$basic_string@DU?$char_traits@D@std@@V?$allocator@D@2@@std@@@?$_List_node_emplace_op2@V?$allocator@U?$_List_node@V?$basic_string@DU?$char_traits@D@std@@V?$allocator@D@2@@std@@PAX@std@@@std@@@std@@QAE@AAV?$allocator@U?$_List_node@V?$basic_string@DU?$char_traits@D@std@@V?$allocator@D@2@@std@@PAX@std@@@1@$$QAV?$basic_string@DU?$char_traits@D@std@@V?$allocator@D@2@@1@@Z$0 0040d670 f   MessageHistory.obj
 0001:0000c67d       __ehhandler$??$?0V?$basic_string@DU?$char_traits@D@std@@V?$allocator@D@2@@std@@@?$_List_node_emplace_op2@V?$allocator@U?$_List_node@V?$basic_string@DU?$char_traits@D@std@@V?$allocator@D@2@@std@@PAX@std@@@std@@@std@@QAE@AAV?$allocator@U?$_List_node@V?$basic_string@DU?$char_traits@D@std@@V?$allocator@D@2@@std@@PAX@std@@@1@$$QAV?$basic_string@DU?$char_traits@D@std@@V?$allocator@D@2@@1@@Z 0040d67d f   MessageHistory.obj
 0001:0000c6a0       __ehhandler$??$_Deallocate@$07$0A@@std@@YAXPAXI@Z 0040d6a0 f   MessageHistory.obj
 0001:0000c6a0       __ehhandler$??$_Freenode0@V?$allocator@U?$_List_node@V?$basic_string@DU?$char_traits@D@std@@V?$allocator@D@2@@std@@PAX@std@@@std@@@?$_List_node@V?$basic_string@DU?$char_traits@D@std@@V?$allocator@D@2@@std@@PAX@std@@SAXAAV?$allocator@U?$_List_node@V?$basic_string@DU?$char_traits@D@std@@V?$allocator@D@2@@std@@PAX@std@@@1@PAU01@@Z 0040d6a0 f   MessageHistory.obj
 0001:0000c6a0       __ehhandler$??$_Freenode@V?$allocator@U?$_List_node@V?$basic_string@DU?$char_traits@D@std@@V?$allocator@D@2@@std@@PAX@std@@@std@@@?$_List_node@V?$basic_string@DU?$char_traits@D@std@@V?$allocator@D@2@@std@@PAX@std@@SAXAAV?$allocator@U?$_List_node@V?$basic_string@DU?$char_traits@D@std@@V?$allocator@D@2@@std@@PAX@std@@@1@PAU01@@Z 0040d6a0 f   MessageHistory.obj
 0001:0000c6c0       __ehhandler$??0?$basic_string@DU?$char_traits@D@std@@V?$allocator@D@2@@std@@QAE@$$QAV01@@Z 0040d6c0 f   MessageHistory.obj
 0001:0000c6e0       __unwindfunclet$??0?$basic_string@DU?$char_traits@D@std@@V?$allocator@D@2@@std@@QAE@QBD@Z$0 0040d6e0 f   MessageHistory.obj
 0001:0000c6ed       __ehhandler$??0?$basic_string@DU?$char_traits@D@std@@V?$allocator@D@2@@std@@QAE@QBD@Z 0040d6ed f   MessageHistory.obj
 0001:0000c710       __ehhandler$??1?$_Alloc_construct_ptr@V?$allocator@U?$_List_node@V?$basic_string@DU?$char_traits@D@std@@V?$allocator@D@2@@std@@PAX@std@@@std@@@std@@QAE@XZ 0040d710 f   MessageHistory.obj
 0001:0000c710       __ehhandler$??1?$_List_node_emplace_op2@V?$allocator@U?$_List_node@V?$basic_string@DU?$char_traits@D@std@@V?$allocator@D@2@@std@@PAX@std@@@std@@@std@@QAE@XZ 0040d710 f   MessageHistory.obj
 0001:0000c730       __ehhandler$?_Tidy_deallocate@?$basic_string@DU?$char_traits@D@std@@V?$allocator@D@2@@std@@AAEXXZ 0040d730 f   MessageHistory.obj
 0001:0000c750       ??__Fg_MessageHistory@@YAXXZ 0040d750 f   jaccessinspector.obj
 0002:00000234       ?pre_cpp_initializer@@3P6AXXZA 0040e234     MSVCRT:exe_winmain.obj
 0002:00000238       ?g_MessageHistory$initializer$@@3P6AXXZA 0040e238     jaccessinspector.obj
 0002:00000244       ?pre_c_initializer@@3P6AHXZA 0040e244     MSVCRT:exe_winmain.obj
 0002:00000248       ?post_pgo_initializer@@3P6AHXZA 0040e248     MSVCRT:exe_winmain.obj
 0002:0000024c       ?__scrt_initialize_tss_var@@3P6AHXZA 0040e24c     MSVCRT:thread_safe_statics.obj
 0002:00000270       $SG43602                   0040e270     AccessBridgeDebug.obj
 0002:0000028c       $SG43604                   0040e28c     AccessBridgeDebug.obj
 0002:00000294       $SG43605                   0040e294     AccessBridgeDebug.obj
 0002:00000298       $SG43607                   0040e298     AccessBridgeDebug.obj
 0002:000002a0       $SG43608                   0040e2a0     AccessBridgeDebug.obj
 0002:000002b8       $SG43635                   0040e2b8     AccessBridgeDebug.obj
 0002:000002d4       $SG43636                   0040e2d4     AccessBridgeDebug.obj
 0002:000002e0       $SG43638                   0040e2e0     AccessBridgeDebug.obj
 0002:000002e4       $SG43680                   0040e2e4     AccessBridgeDebug.obj
 0002:000002ec       $SG43681                   0040e2ec     AccessBridgeDebug.obj
 0002:000002f0       $SG43697                   0040e2f0     AccessBridgeDebug.obj
 0002:000002f8       $SG43698                   0040e2f8     AccessBridgeDebug.obj
 0002:000002fc       $SG43740                   0040e2fc     AccessBridgeDebug.obj
 0002:00000304       $SG43741                   0040e304     AccessBridgeDebug.obj
 0002:00000308       $SG43757                   0040e308     AccessBridgeDebug.obj
 0002:00000310       $SG43758                   0040e310     AccessBridgeDebug.obj
 0002:00000314       $SG38458                   0040e314     AccessBridgeMessages.obj
 0002:00000330       $SG38459                   0040e330     AccessBridgeMessages.obj
 0002:00000350       $SG47878                   0040e350     AccessInfo.obj
 0002:00000354       $SG47880                   0040e354     AccessInfo.obj
 0002:00000358       $SG47883                   0040e358     AccessInfo.obj
 0002:00000364       $SG47928                   0040e364     AccessInfo.obj
 0002:00000390       $SG47929                   0040e390     AccessInfo.obj
 0002:00000394       $SG47930                   0040e394     AccessInfo.obj
 0002:00000398       $SG47948                   0040e398     AccessInfo.obj
 0002:0000039c       $SG48090                   0040e39c     AccessInfo.obj
 0002:000003c4       $SG48091                   0040e3c4     AccessInfo.obj
 0002:000003dc       $SG48092                   0040e3dc     AccessInfo.obj
 0002:00000404       $SG48093                   0040e404     AccessInfo.obj
 0002:00000430       $SG48094                   0040e430     AccessInfo.obj
 0002:0000045c       $SG48095                   0040e45c     AccessInfo.obj
 0002:0000048c       $SG48099                   0040e48c     AccessInfo.obj
 0002:000004b8       $SG48100                   0040e4b8     AccessInfo.obj
 0002:000004dc       $SG48103                   0040e4dc     AccessInfo.obj
 0002:000004f8       $SG48104                   0040e4f8     AccessInfo.obj
 0002:000004fc       $SG48105                   0040e4fc     AccessInfo.obj
 0002:00000510       $SG48108                   0040e510     AccessInfo.obj
 0002:00000534       $SG48109                   0040e534     AccessInfo.obj
 0002:00000550       $SG48110                   0040e550     AccessInfo.obj
 0002:00000568       $SG48111                   0040e568     AccessInfo.obj
 0002:0000057c       $SG48112                   0040e57c     AccessInfo.obj
 0002:000005a0       $SG48113                   0040e5a0     AccessInfo.obj
 0002:000005b4       $SG48114                   0040e5b4     AccessInfo.obj
 0002:000005d8       $SG48115                   0040e5d8     AccessInfo.obj
 0002:000005f4       $SG48116                   0040e5f4     AccessInfo.obj
 0002:00000610       $SG48117                   0040e610     AccessInfo.obj
 0002:0000063c       $SG48120                   0040e63c     AccessInfo.obj
 0002:00000660       $SG48123                   0040e660     AccessInfo.obj
 0002:000006a0       $SG48126                   0040e6a0     AccessInfo.obj
 0002:000006c4       $SG48127                   0040e6c4     AccessInfo.obj
 0002:000006e8       $SG48128                   0040e6e8     AccessInfo.obj
 0002:0000070c       $SG48131                   0040e70c     AccessInfo.obj
 0002:0000071c       $SG48134                   0040e71c     AccessInfo.obj
 0002:00000750       $SG48135                   0040e750     AccessInfo.obj
 0002:00000768       $SG48138                   0040e768     AccessInfo.obj
 0002:0000078c       $SG48139                   0040e78c     AccessInfo.obj
 0002:000007ac       $SG48140                   0040e7ac     AccessInfo.obj
 0002:000007c4       $SG48143                   0040e7c4     AccessInfo.obj
 0002:000007ec       $SG48144                   0040e7ec     AccessInfo.obj
 0002:00000814       $SG48148                   0040e814     AccessInfo.obj
 0002:00000838       $SG48152                   0040e838     AccessInfo.obj
 0002:0000085c       $SG48153                   0040e85c     AccessInfo.obj
 0002:0000087c       $SG48154                   0040e87c     AccessInfo.obj
 0002:0000089c       $SG48156                   0040e89c     AccessInfo.obj
 0002:000008c4       $SG48158                   0040e8c4     AccessInfo.obj
 0002:000008e0       $SG48161                   0040e8e0     AccessInfo.obj
 0002:00000924       $SG48164                   0040e924     AccessInfo.obj
 0002:00000960       $SG48167                   0040e960     AccessInfo.obj
 0002:00000984       $SG48168                   0040e984     AccessInfo.obj
 0002:000009a4       $SG48169                   0040e9a4     AccessInfo.obj
 0002:000009c4       $SG48170                   0040e9c4     AccessInfo.obj
 0002:000009f0       $SG48172                   0040e9f0     AccessInfo.obj
 0002:00000a10       $SG48173                   0040ea10     AccessInfo.obj
 0002:00000a34       $SG48174                   0040ea34     AccessInfo.obj
 0002:00000a58       $SG48175                   0040ea58     AccessInfo.obj
 0002:00000a7c       $SG48177                   0040ea7c     AccessInfo.obj
 0002:00000a98       $SG48178                   0040ea98     AccessInfo.obj
 0002:00000ab4       $SG48179                   0040eab4     AccessInfo.obj
 0002:00000ad4       $SG48180                   0040ead4     AccessInfo.obj
 0002:00000af0       $SG48181                   0040eaf0     AccessInfo.obj
 0002:00000b08       $SG48183                   0040eb08     AccessInfo.obj
 0002:00000b24       $SG48184                   0040eb24     AccessInfo.obj
 0002:00000b44       $SG48185                   0040eb44     AccessInfo.obj
 0002:00000b60       $SG48188                   0040eb60     AccessInfo.obj
 0002:00000b84       $SG48190                   0040eb84     AccessInfo.obj
 0002:00000bac       $SG48191                   0040ebac     AccessInfo.obj
 0002:00000bcc       $SG48192                   0040ebcc     AccessInfo.obj
 0002:00000be8       $SG48193                   0040ebe8     AccessInfo.obj
 0002:00000c0c       $SG48196                   0040ec0c     AccessInfo.obj
 0002:00000c38       $SG48199                   0040ec38     AccessInfo.obj
 0002:00000c5c       $SG48200                   0040ec5c     AccessInfo.obj
 0002:00000c7c       $SG48201                   0040ec7c     AccessInfo.obj
 0002:00000c9c       $SG48203                   0040ec9c     AccessInfo.obj
 0002:00000cc0       $SG48205                   0040ecc0     AccessInfo.obj
 0002:00000cdc       $SG48207                   0040ecdc     AccessInfo.obj
 0002:00000cf8       $SG48209                   0040ecf8     AccessInfo.obj
 0002:00000d14       $SG48213                   0040ed14     AccessInfo.obj
 0002:00000d3c       $SG48214                   0040ed3c     AccessInfo.obj
 0002:00000d58       $SG48215                   0040ed58     AccessInfo.obj
 0002:00000d7c       $SG48216                   0040ed7c     AccessInfo.obj
 0002:00000da0       $SG48217                   0040eda0     AccessInfo.obj
 0002:00000dc4       $SG48218                   0040edc4     AccessInfo.obj
 0002:00000de0       $SG48219                   0040ede0     AccessInfo.obj
 0002:00000e00       $SG48222                   0040ee00     AccessInfo.obj
 0002:00000e2c       $SG48223                   0040ee2c     AccessInfo.obj
 0002:00000e58       $SG48224                   0040ee58     AccessInfo.obj
 0002:00000e6c       $SG48225                   0040ee6c     AccessInfo.obj
 0002:00000e84       $SG48226                   0040ee84     AccessInfo.obj
 0002:00000ea0       $SG48227                   0040eea0     AccessInfo.obj
 0002:00000eb8       $SG48230                   0040eeb8     AccessInfo.obj
 0002:00000efc       $SG48233                   0040eefc     AccessInfo.obj
 0002:00000f20       $SG48234                   0040ef20     AccessInfo.obj
 0002:00000f34       $SG48235                   0040ef34     AccessInfo.obj
 0002:00000f48       $SG48238                   0040ef48     AccessInfo.obj
 0002:00000f78       $SG48239                   0040ef78     AccessInfo.obj
 0002:00000fa0       $SG48240                   0040efa0     AccessInfo.obj
 0002:00000fc4       $SG48241                   0040efc4     AccessInfo.obj
 0002:00000fec       $SG48242                   0040efec     AccessInfo.obj
 0002:0000100c       $SG48245                   0040f00c     AccessInfo.obj
 0002:00001040       $SG48246                   0040f040     AccessInfo.obj
 0002:00001058       $SG48247                   0040f058     AccessInfo.obj
 0002:0000105c       $SG48250                   0040f05c     AccessInfo.obj
 0002:00001088       $SG48251                   0040f088     AccessInfo.obj
 0002:000010ac       $SG48252                   0040f0ac     AccessInfo.obj
 0002:000010c0       $SG48253                   0040f0c0     AccessInfo.obj
 0002:000010d8       $SG48254                   0040f0d8     AccessInfo.obj
 0002:000010f4       $SG48255                   0040f0f4     AccessInfo.obj
 0002:0000110c       $SG48258                   0040f10c     AccessInfo.obj
 0002:00001138       $SG48261                   0040f138     AccessInfo.obj
 0002:0000115c       $SG48262                   0040f15c     AccessInfo.obj
 0002:00001170       $SG48263                   0040f170     AccessInfo.obj
 0002:00001184       $SG48265                   0040f184     AccessInfo.obj
 0002:000011a8       $SG48267                   0040f1a8     AccessInfo.obj
 0002:000011d0       $SG48268                   0040f1d0     AccessInfo.obj
 0002:000011f0       $SG48269                   0040f1f0     AccessInfo.obj
 0002:00001208       $SG48271                   0040f208     AccessInfo.obj
 0002:0000122c       $SG48272                   0040f22c     AccessInfo.obj
 0002:0000124c       $SG48273                   0040f24c     AccessInfo.obj
 0002:00001268       $SG48274                   0040f268     AccessInfo.obj
 0002:0000128c       $SG48276                   0040f28c     AccessInfo.obj
 0002:000012c8       $SG48279                   0040f2c8     AccessInfo.obj
 0002:000012e8       $SG48281                   0040f2e8     AccessInfo.obj
 0002:00001304       $SG48282                   0040f304     AccessInfo.obj
 0002:0000131c       $SG48283                   0040f31c     AccessInfo.obj
 0002:00001338       $SG48285                   0040f338     AccessInfo.obj
 0002:00001340       $SG48286                   0040f340     AccessInfo.obj
 0002:0000134c       $SG48287                   0040f34c     AccessInfo.obj
 0002:0000136c       $SG48288                   0040f36c     AccessInfo.obj
 0002:00001374       $SG48289                   0040f374     AccessInfo.obj
 0002:00001380       $SG48290                   0040f380     AccessInfo.obj
 0002:00001388       $SG48291                   0040f388     AccessInfo.obj
 0002:00001394       $SG48292                   0040f394     AccessInfo.obj
 0002:000013a4       $SG48293                   0040f3a4     AccessInfo.obj
 0002:000013ac       $SG48294                   0040f3ac     AccessInfo.obj
 0002:000013bc       $SG48295                   0040f3bc     AccessInfo.obj
 0002:000013d0       $SG48296                   0040f3d0     AccessInfo.obj
 0002:000013d8       $SG48297                   0040f3d8     AccessInfo.obj
 0002:000013e4       $SG48298                   0040f3e4     AccessInfo.obj
 0002:000013f4       $SG48299                   0040f3f4     AccessInfo.obj
 0002:000013fc       $SG48300                   0040f3fc     AccessInfo.obj
 0002:00001408       $SG48301                   0040f408     AccessInfo.obj
 0002:00001418       $SG48302                   0040f418     AccessInfo.obj
 0002:00001420       $SG48303                   0040f420     AccessInfo.obj
 0002:00001444       $SG48304                   0040f444     AccessInfo.obj
 0002:00001468       $SG48305                   0040f468     AccessInfo.obj
 0002:00001484       $SG48306                   0040f484     AccessInfo.obj
 0002:000014a0       $SG48307                   0040f4a0     AccessInfo.obj
 0002:000014c4       $SG48308                   0040f4c4     AccessInfo.obj
 0002:000014e0       $SG48309                   0040f4e0     AccessInfo.obj
 0002:000014fc       $SG48310                   0040f4fc     AccessInfo.obj
 0002:00001518       $SG48311                   0040f518     AccessInfo.obj
 0002:00001534       $SG48312                   0040f534     AccessInfo.obj
 0002:00001550       $SG48313                   0040f550     AccessInfo.obj
 0002:00001578       $SG48316                   0040f578     AccessInfo.obj
 0002:00001598       $SG48317                   0040f598     AccessInfo.obj
 0002:000015c4       $SG48318                   0040f5c4     AccessInfo.obj
 0002:000015e0       $SG48320                   0040f5e0     AccessInfo.obj
 0002:00001618       $SG48322                   0040f618     AccessInfo.obj
 0002:00001654       $SG48325                   0040f654     AccessInfo.obj
 0002:00001674       $SG48327                   0040f674     AccessInfo.obj
 0002:00001690       $SG48328                   0040f690     AccessInfo.obj
 0002:000016a8       $SG48329                   0040f6a8     AccessInfo.obj
 0002:000016c4       $SG48331                   0040f6c4     AccessInfo.obj
 0002:000016cc       $SG48332                   0040f6cc     AccessInfo.obj
 0002:000016d8       $SG48333                   0040f6d8     AccessInfo.obj
 0002:000016f8       $SG48334                   0040f6f8     AccessInfo.obj
 0002:00001700       $SG48335                   0040f700     AccessInfo.obj
 0002:0000170c       $SG48336                   0040f70c     AccessInfo.obj
 0002:00001714       $SG48337                   0040f714     AccessInfo.obj
 0002:00001720       $SG48338                   0040f720     AccessInfo.obj
 0002:00001730       $SG48339                   0040f730     AccessInfo.obj
 0002:00001738       $SG48340                   0040f738     AccessInfo.obj
 0002:00001748       $SG48341                   0040f748     AccessInfo.obj
 0002:0000175c       $SG48342                   0040f75c     AccessInfo.obj
 0002:00001764       $SG48343                   0040f764     AccessInfo.obj
 0002:00001770       $SG48344                   0040f770     AccessInfo.obj
 0002:00001780       $SG48345                   0040f780     AccessInfo.obj
 0002:00001788       $SG48346                   0040f788     AccessInfo.obj
 0002:00001794       $SG48347                   0040f794     AccessInfo.obj
 0002:000017a4       $SG48348                   0040f7a4     AccessInfo.obj
 0002:000017ac       $SG48349                   0040f7ac     AccessInfo.obj
 0002:000017d0       $SG48350                   0040f7d0     AccessInfo.obj
 0002:000017f4       $SG48351                   0040f7f4     AccessInfo.obj
 0002:00001810       $SG48352                   0040f810     AccessInfo.obj
 0002:0000182c       $SG48353                   0040f82c     AccessInfo.obj
 0002:00001850       $SG48354                   0040f850     AccessInfo.obj
 0002:0000186c       $SG48355                   0040f86c     AccessInfo.obj
 0002:00001888       $SG48356                   0040f888     AccessInfo.obj
 0002:000018a4       $SG48357                   0040f8a4     AccessInfo.obj
 0002:000018c0       $SG48358                   0040f8c0     AccessInfo.obj
 0002:000018dc       $SG48359                   0040f8dc     AccessInfo.obj
 0002:00001904       $SG48362                   0040f904     AccessInfo.obj
 0002:00001924       $SG48363                   0040f924     AccessInfo.obj
 0002:0000194d       $SG59989                   0040f94d     MessageHistory.obj
 0002:0000194e       $SG59995                   0040f94e     MessageHistory.obj
 0002:0000194f       $SG60002                   0040f94f     MessageHistory.obj
 0002:00001950       $SG60009                   0040f950     MessageHistory.obj
 0002:00001951       $SG60031                   0040f951     MessageHistory.obj
 0002:00001952       $SG60045                   0040f952     MessageHistory.obj
 0002:00001953       $SG60047                   0040f953     MessageHistory.obj
 0002:000019c8       $SG66335                   0040f9c8     jaccessinspector.obj
 0002:000019cc       $SG66336                   0040f9cc     jaccessinspector.obj
 0002:000019e4       $SG66337                   0040f9e4     jaccessinspector.obj
 0002:00001a08       $SG66338                   0040fa08     jaccessinspector.obj
 0002:00001a1c       $SG66404                   0040fa1c     jaccessinspector.obj
 0002:00001a38       $SG66412                   0040fa38     jaccessinspector.obj
 0002:00001a48       $SG66421                   0040fa48     jaccessinspector.obj
 0002:00001a58       $SG66516                   0040fa58     jaccessinspector.obj
 0002:00001a88       $SG66527                   0040fa88     jaccessinspector.obj
 0002:00001abc       $SG66538                   0040fabc     jaccessinspector.obj
 0002:00001aec       $SG66549                   0040faec     jaccessinspector.obj
 0002:00001b1c       $SG66558                   0040fb1c     jaccessinspector.obj
 0002:00001b38       $SG66566                   0040fb38     jaccessinspector.obj
 0002:00001b50       $SG66576                   0040fb50     jaccessinspector.obj
 0002:00001b8c       $SG66585                   0040fb8c     jaccessinspector.obj
 0002:00001bac       $SG66600                   0040fbac     jaccessinspector.obj
 0002:00001be8       $SG66602                   0040fbe8     jaccessinspector.obj
 0002:00001c08       $SG66603                   0040fc08     jaccessinspector.obj
 0002:00001c10       $SG66605                   0040fc10     jaccessinspector.obj
 0002:00001c30       $SG66606                   0040fc30     jaccessinspector.obj
 0002:00001c38       $SG66617                   0040fc38     jaccessinspector.obj
 0002:00001c80       $SG66628                   0040fc80     jaccessinspector.obj
 0002:00001cb0       $SG66927                   0040fcb0     jaccessinspector.obj
 0002:00001cbc       $SG66929                   0040fcbc     jaccessinspector.obj
 0002:00001cd0       $SG66931                   0040fcd0     jaccessinspector.obj
 0002:00001ce4       $SG66933                   0040fce4     jaccessinspector.obj
 0002:00001cf8       $SG66935                   0040fcf8     jaccessinspector.obj
 0002:00001d0c       $SG66937                   0040fd0c     jaccessinspector.obj
 0002:00001d1c       $SG66939                   0040fd1c     jaccessinspector.obj
 0002:00001d28       $SG66941                   0040fd28     jaccessinspector.obj
 0002:00001d38       $SG66943                   0040fd38     jaccessinspector.obj
 0002:00001d44       $SG66945                   0040fd44     jaccessinspector.obj
 0002:00001d58       $SG66947                   0040fd58     jaccessinspector.obj
 0002:00001d6c       $SG66949                   0040fd6c     jaccessinspector.obj
 0002:00001d80       $SG66951                   0040fd80     jaccessinspector.obj
 0002:00001d94       $SG66953                   0040fd94     jaccessinspector.obj
 0002:00001da8       $SG66955                   0040fda8     jaccessinspector.obj
 0002:00001dbc       $SG66957                   0040fdbc     jaccessinspector.obj
 0002:00001dd4       $SG66959                   0040fdd4     jaccessinspector.obj
 0002:00001df4       $SG66961                   0040fdf4     jaccessinspector.obj
 0002:00001e10       $SG66963                   0040fe10     jaccessinspector.obj
 0002:00001e2c       $SG66965                   0040fe2c     jaccessinspector.obj
 0002:00001e4c       $SG66967                   0040fe4c     jaccessinspector.obj
 0002:00001e64       $SG66969                   0040fe64     jaccessinspector.obj
 0002:00001e80       $SG66971                   0040fe80     jaccessinspector.obj
 0002:00001ea0       $SG66973                   0040fea0     jaccessinspector.obj
 0002:00001ebc       $SG66975                   0040febc     jaccessinspector.obj
 0002:00001ee0       $SG66977                   0040fee0     jaccessinspector.obj
 0002:00001f00       $SG67072                   0040ff00     jaccessinspector.obj
 0002:00001f0c       $SG67075                   0040ff0c     jaccessinspector.obj
 0002:00001f20       $SG67078                   0040ff20     jaccessinspector.obj
 0002:00001f34       $SG67081                   0040ff34     jaccessinspector.obj
 0002:00001f48       $SG67084                   0040ff48     jaccessinspector.obj
 0002:00001f5c       $SG67087                   0040ff5c     jaccessinspector.obj
 0002:00001f6c       $SG67090                   0040ff6c     jaccessinspector.obj
 0002:00001f78       $SG67093                   0040ff78     jaccessinspector.obj
 0002:00001f88       $SG67096                   0040ff88     jaccessinspector.obj
 0002:00001f94       $SG67099                   0040ff94     jaccessinspector.obj
 0002:00001fa8       $SG67102                   0040ffa8     jaccessinspector.obj
 0002:00001fbc       $SG67105                   0040ffbc     jaccessinspector.obj
 0002:00001fd0       $SG67108                   0040ffd0     jaccessinspector.obj
 0002:00001fe4       $SG67111                   0040ffe4     jaccessinspector.obj
 0002:00001ff8       $SG67114                   0040fff8     jaccessinspector.obj
 0002:0000200c       $SG67117                   0041000c     jaccessinspector.obj
 0002:00002024       $SG67120                   00410024     jaccessinspector.obj
 0002:00002044       $SG67123                   00410044     jaccessinspector.obj
 0002:00002060       $SG67126                   00410060     jaccessinspector.obj
 0002:0000207c       $SG67129                   0041007c     jaccessinspector.obj
 0002:0000209c       $SG67132                   0041009c     jaccessinspector.obj
 0002:000020b4       $SG67135                   004100b4     jaccessinspector.obj
 0002:000020d0       $SG67138                   004100d0     jaccessinspector.obj
 0002:000020f0       $SG67141                   004100f0     jaccessinspector.obj
 0002:0000210c       $SG67144                   0041010c     jaccessinspector.obj
 0002:00002130       $SG67147                   00410130     jaccessinspector.obj
 0002:00002150       $SG67245                   00410150     jaccessinspector.obj
 0002:0000215c       ?jaccessinspectorOptionsRegistryKey@@3QBDB 0041015c     jaccessinspector.obj
 0002:00002160       $SG48002                   00410160     jaccessinspector.obj
 0002:00002198       _GS_ExceptionPointers      00410198     MSVCRT:gs_report.obj
 0002:000028a8       __unwindtable$??0?$basic_string@DU?$char_traits@D@std@@V?$allocator@D@2@@std@@QAE@QBD@Z 004108a8     MessageHistory.obj
 0002:000028b0       __ehfuncinfo$??0?$basic_string@DU?$char_traits@D@std@@V?$allocator@D@2@@std@@QAE@QBD@Z 004108b0     MessageHistory.obj
 0002:000028d4       __ehfuncinfo$??$_Deallocate@$07$0A@@std@@YAXPAXI@Z 004108d4     MessageHistory.obj
 0002:000028d4       __ehfuncinfo$??$_Freenode0@V?$allocator@U?$_List_node@V?$basic_string@DU?$char_traits@D@std@@V?$allocator@D@2@@std@@PAX@std@@@std@@@?$_List_node@V?$basic_string@DU?$char_traits@D@std@@V?$allocator@D@2@@std@@PAX@std@@SAXAAV?$allocator@U?$_List_node@V?$basic_string@DU?$char_traits@D@std@@V?$allocator@D@2@@std@@PAX@std@@@1@PAU01@@Z 004108d4     MessageHistory.obj
 0002:000028d4       __ehfuncinfo$??$_Freenode@V?$allocator@U?$_List_node@V?$basic_string@DU?$char_traits@D@std@@V?$allocator@D@2@@std@@PAX@std@@@std@@@?$_List_node@V?$basic_string@DU?$char_traits@D@std@@V?$allocator@D@2@@std@@PAX@std@@SAXAAV?$allocator@U?$_List_node@V?$basic_string@DU?$char_traits@D@std@@V?$allocator@D@2@@std@@PAX@std@@@1@PAU01@@Z 004108d4     MessageHistory.obj
 0002:000028d4       __ehfuncinfo$??0?$basic_string@DU?$char_traits@D@std@@V?$allocator@D@2@@std@@QAE@$$QAV01@@Z 004108d4     MessageHistory.obj
 0002:000028d4       __ehfuncinfo$??1?$_Alloc_construct_ptr@V?$allocator@U?$_List_node@V?$basic_string@DU?$char_traits@D@std@@V?$allocator@D@2@@std@@PAX@std@@@std@@@std@@QAE@XZ 004108d4     MessageHistory.obj
 0002:000028d4       __ehfuncinfo$??1?$_List_node_emplace_op2@V?$allocator@U?$_List_node@V?$basic_string@DU?$char_traits@D@std@@V?$allocator@D@2@@std@@PAX@std@@@std@@@std@@QAE@XZ 004108d4     MessageHistory.obj
 0002:000028d4       __ehfuncinfo$?_Tidy_deallocate@?$basic_string@DU?$char_traits@D@std@@V?$allocator@D@2@@std@@AAEXXZ 004108d4     MessageHistory.obj
 0002:000028f8       __unwindtable$?AddMessage@MessageHistory@@QAEXPBD@Z 004108f8     MessageHistory.obj
 0002:00002900       __ehfuncinfo$?AddMessage@MessageHistory@@QAEXPBD@Z 00410900     MessageHistory.obj
 0002:00002924       __unwindtable$??$?0V?$basic_string@DU?$char_traits@D@std@@V?$allocator@D@2@@std@@@?$_List_node_emplace_op2@V?$allocator@U?$_List_node@V?$basic_string@DU?$char_traits@D@std@@V?$allocator@D@2@@std@@PAX@std@@@std@@@std@@QAE@AAV?$allocator@U?$_List_node@V?$basic_string@DU?$char_traits@D@std@@V?$allocator@D@2@@std@@PAX@std@@@1@$$QAV?$basic_string@DU?$char_traits@D@std@@V?$allocator@D@2@@1@@Z 00410924     MessageHistory.obj
 0002:0000292c       __ehfuncinfo$??$?0V?$basic_string@DU?$char_traits@D@std@@V?$allocator@D@2@@std@@@?$_List_node_emplace_op2@V?$allocator@U?$_List_node@V?$basic_string@DU?$char_traits@D@std@@V?$allocator@D@2@@std@@PAX@std@@@std@@@std@@QAE@AAV?$allocator@U?$_List_node@V?$basic_string@DU?$char_traits@D@std@@V?$allocator@D@2@@std@@PAX@std@@@1@$$QAV?$basic_string@DU?$char_traits@D@std@@V?$allocator@D@2@@1@@Z 0041092c     MessageHistory.obj
 0002:000029c8       __sehtable$___scrt_is_nonwritable_in_current_image 004109c8     MSVCRT:utility.obj
 0002:000029e8       __sehtable$?__scrt_common_main_seh@@YAHXZ 004109e8     MSVCRT:exe_winmain.obj
 0002:00002dc8       .idata$6                   00410dc8     advapi32:ADVAPI32.dll
 0002:00003068       .idata$6                   00411068     user32:USER32.dll
 0002:00003094       .idata$6                   00411094     msvcprt:MSVCP140.dll
 0002:000032ee       .idata$6                   004112ee     kernel32:KERNEL32.dll
 0002:000033c6       .idata$6                   004113c6     vcruntime:VCRUNTIME140.dll
 0002:00003698       .idata$6                   00411698     ucrt:api-ms-win-crt-string-l1-1-0.dll
 0002:000036ba       .idata$6                   004116ba     ucrt:api-ms-win-crt-stdio-l1-1-0.dll
 0002:000036da       .idata$6                   004116da     ucrt:api-ms-win-crt-environment-l1-1-0.dll
 0002:00003700       .idata$6                   00411700     ucrt:api-ms-win-crt-time-l1-1-0.dll
 0002:00003720       .idata$6                   00411720     ucrt:api-ms-win-crt-runtime-l1-1-0.dll
 0002:00003742       .idata$6                   00411742     ucrt:api-ms-win-crt-heap-l1-1-0.dll
 0002:00003762       .idata$6                   00411762     ucrt:api-ms-win-crt-math-l1-1-0.dll
 0002:00003782       .idata$6                   00411782     ucrt:api-ms-win-crt-locale-l1-1-0.dll
 0003:00000000       $SG46443                   00412000     AccessBridgeCalls.obj
 0003:00000014       $SG46447                   00412014     AccessBridgeCalls.obj
 0003:00000020       $SG46449                   00412020     AccessBridgeCalls.obj
 0003:00000034       $SG46451                   00412034     AccessBridgeCalls.obj
 0003:00000048       $SG46453                   00412048     AccessBridgeCalls.obj
 0003:00000058       $SG46455                   00412058     AccessBridgeCalls.obj
 0003:0000006c       $SG46457                   0041206c     AccessBridgeCalls.obj
 0003:00000080       $SG46459                   00412080     AccessBridgeCalls.obj
 0003:00000094       $SG46461                   00412094     AccessBridgeCalls.obj
 0003:000000a8       $SG46463                   004120a8     AccessBridgeCalls.obj
 0003:000000bc       $SG46465                   004120bc     AccessBridgeCalls.obj
 0003:000000d0       $SG46467                   004120d0     AccessBridgeCalls.obj
 0003:000000e4       $SG46469                   004120e4     AccessBridgeCalls.obj
 0003:000000f8       $SG46471                   004120f8     AccessBridgeCalls.obj
 0003:0000010c       $SG46473                   0041210c     AccessBridgeCalls.obj
 0003:00000124       $SG46475                   00412124     AccessBridgeCalls.obj
 0003:00000148       $SG46477                   00412148     AccessBridgeCalls.obj
 0003:00000168       $SG46479                   00412168     AccessBridgeCalls.obj
 0003:00000180       $SG46481                   00412180     AccessBridgeCalls.obj
 0003:000001a0       $SG46483                   004121a0     AccessBridgeCalls.obj
 0003:000001bc       $SG46485                   004121bc     AccessBridgeCalls.obj
 0003:000001d8       $SG46487                   004121d8     AccessBridgeCalls.obj
 0003:000001f8       $SG46489                   004121f8     AccessBridgeCalls.obj
 0003:00000210       $SG46491                   00412210     AccessBridgeCalls.obj
 0003:0000022c       $SG46493                   0041222c     AccessBridgeCalls.obj
 0003:0000024c       $SG46495                   0041224c     AccessBridgeCalls.obj
 0003:00000268       $SG46497                   00412268     AccessBridgeCalls.obj
 0003:0000028c       $SG46499                   0041228c     AccessBridgeCalls.obj
 0003:000002ac       $SG46501                   004122ac     AccessBridgeCalls.obj
 0003:000002c0       $SG46503                   004122c0     AccessBridgeCalls.obj
 0003:000002d0       $SG46505                   004122d0     AccessBridgeCalls.obj
 0003:000002e0       $SG46507                   004122e0     AccessBridgeCalls.obj
 0003:000002f0       $SG46509                   004122f0     AccessBridgeCalls.obj
 0003:00000310       $SG46511                   00412310     AccessBridgeCalls.obj
 0003:00000330       $SG46513                   00412330     AccessBridgeCalls.obj
 0003:00000348       $SG46515                   00412348     AccessBridgeCalls.obj
 0003:00000368       $SG46517                   00412368     AccessBridgeCalls.obj
 0003:00000384       $SG46519                   00412384     AccessBridgeCalls.obj
 0003:000003a4       $SG46521                   004123a4     AccessBridgeCalls.obj
 0003:000003c4       $SG46523                   004123c4     AccessBridgeCalls.obj
 0003:000003dc       $SG46525                   004123dc     AccessBridgeCalls.obj
 0003:000003f8       $SG46527                   004123f8     AccessBridgeCalls.obj
 0003:00000414       $SG46529                   00412414     AccessBridgeCalls.obj
 0003:00000434       $SG46531                   00412434     AccessBridgeCalls.obj
 0003:00000458       $SG46533                   00412458     AccessBridgeCalls.obj
 0003:0000047c       $SG46535                   0041247c     AccessBridgeCalls.obj
 0003:000004a0       $SG46537                   004124a0     AccessBridgeCalls.obj
 0003:000004c0       $SG46539                   004124c0     AccessBridgeCalls.obj
 0003:000004e0       $SG46541                   004124e0     AccessBridgeCalls.obj
 0003:00000508       $SG46543                   00412508     AccessBridgeCalls.obj
 0003:00000528       $SG46545                   00412528     AccessBridgeCalls.obj
 0003:0000054c       $SG46547                   0041254c     AccessBridgeCalls.obj
 0003:00000564       $SG46549                   00412564     AccessBridgeCalls.obj
 0003:00000580       $SG46551                   00412580     AccessBridgeCalls.obj
 0003:00000598       $SG46553                   00412598     AccessBridgeCalls.obj
 0003:000005b4       $SG46555                   004125b4     AccessBridgeCalls.obj
 0003:000005cc       $SG46557                   004125cc     AccessBridgeCalls.obj
 0003:000005e8       $SG46559                   004125e8     AccessBridgeCalls.obj
 0003:00000604       $SG46561                   00412604     AccessBridgeCalls.obj
 0003:00000620       $SG46563                   00412620     AccessBridgeCalls.obj
 0003:00000640       $SG46565                   00412640     AccessBridgeCalls.obj
 0003:00000658       $SG46567                   00412658     AccessBridgeCalls.obj
 0003:00000674       $SG46569                   00412674     AccessBridgeCalls.obj
 0003:00000688       $SG46571                   00412688     AccessBridgeCalls.obj
 0003:000006a0       $SG46573                   004126a0     AccessBridgeCalls.obj
 0003:000006b4       $SG46575                   004126b4     AccessBridgeCalls.obj
 0003:000006cc       $SG46577                   004126cc     AccessBridgeCalls.obj
 0003:000006e4       $SG46579                   004126e4     AccessBridgeCalls.obj
 0003:00000704       $SG46581                   00412704     AccessBridgeCalls.obj
 0003:00000720       $SG46583                   00412720     AccessBridgeCalls.obj
 0003:00000738       $SG46585                   00412738     AccessBridgeCalls.obj
 0003:00000754       $SG46587                   00412754     AccessBridgeCalls.obj
 0003:0000076c       $SG46589                   0041276c     AccessBridgeCalls.obj
 0003:00000794       $SG46591                   00412794     AccessBridgeCalls.obj
 0003:000007bc       $SG46593                   004127bc     AccessBridgeCalls.obj
 0003:000007e4       $SG46595                   004127e4     AccessBridgeCalls.obj
 0003:00000808       $SG46597                   00412808     AccessBridgeCalls.obj
 0003:0000082c       $SG46599                   0041282c     AccessBridgeCalls.obj
 0003:00000850       $SG46601                   00412850     AccessBridgeCalls.obj
 0003:00000878       $SG46603                   00412878     AccessBridgeCalls.obj
 0003:000008a0       $SG46605                   004128a0     AccessBridgeCalls.obj
 0003:000008c8       $SG46607                   004128c8     AccessBridgeCalls.obj
 0003:000008f0       $SG46609                   004128f0     AccessBridgeCalls.obj
 0003:00000900       $SG46611                   00412900     AccessBridgeCalls.obj
 0003:00000914       $SG46613                   00412914     AccessBridgeCalls.obj
 0003:00000928       $SG46615                   00412928     AccessBridgeCalls.obj
 0003:00000944       $SG46617                   00412944     AccessBridgeCalls.obj
 0003:00000954       $SG46619                   00412954     AccessBridgeCalls.obj
 0003:00000968       $SG46621                   00412968     AccessBridgeCalls.obj
 0003:00000984       $SG46623                   00412984     AccessBridgeCalls.obj
 0003:00000994       $SG46625                   00412994     AccessBridgeCalls.obj
 0003:000009a4       $SG46627                   004129a4     AccessBridgeCalls.obj
 0003:000009c0       $SG46629                   004129c0     AccessBridgeCalls.obj
 0003:000009d8       $SG46631                   004129d8     AccessBridgeCalls.obj
 0003:000009ec       $SG46633                   004129ec     AccessBridgeCalls.obj
 0003:00000a00       $SG46635                   00412a00     AccessBridgeCalls.obj
 0003:00000a14       $SG46637                   00412a14     AccessBridgeCalls.obj
 0003:00000a28       ?warning@?1??appendToBuffer@@YAHPADI0ZZ@4PADA 00412a28     AccessInfo.obj
 0003:00000b30       _logFP                     00412b30     AccessBridgeDebug.obj
 0003:00000b38       ?retbuf@?1??printError@@9@4PADA 00412b38     AccessBridgeDebug.obj
 0003:00000c48       ?datebuf@?1??getTimeAndDate@@YAPADXZ@4PADA 00412c48     AccessInfo.obj
 0003:00000d24       ?titleBarHeight@?1??jaccessinspectorDialogProc@@YGHPAUHWND__@@IIJ@Z@4HA 00412d24     jaccessinspector.obj
 0003:00000d28       ?$TSS0@?1??jaccessinspectorDialogProc@@YGHPAUHWND__@@IIJ@Z@4HA 00412d28     jaccessinspector.obj
 0003:00000d2c       ?menuBarHeight@?1??jaccessinspectorDialogProc@@YGHPAUHWND__@@IIJ@Z@4HA 00412d2c     jaccessinspector.obj
 0003:00000d30       ?$TSS1@?1??jaccessinspectorDialogProc@@YGHPAUHWND__@@IIJ@Z@4HA 00412d30     jaccessinspector.obj
 0003:00000d34       ?borderHeight@?1??jaccessinspectorDialogProc@@YGHPAUHWND__@@IIJ@Z@4HA 00412d34     jaccessinspector.obj
 0003:00000d38       ?$TSS2@?1??jaccessinspectorDialogProc@@YGHPAUHWND__@@IIJ@Z@4HA 00412d38     jaccessinspector.obj
 0003:00000d3c       ?borderWidth@?1??jaccessinspectorDialogProc@@YGHPAUHWND__@@IIJ@Z@4HA 00412d3c     jaccessinspector.obj
 0003:00000d40       ?$TSS3@?1??jaccessinspectorDialogProc@@YGHPAUHWND__@@IIJ@Z@4HA 00412d40     jaccessinspector.obj
 0003:00000d44       ?verticalScrollBarWidth@?1??jaccessinspectorDialogProc@@YGHPAUHWND__@@IIJ@Z@4HA 00412d44     jaccessinspector.obj
 0003:00000d48       ?$TSS4@?1??jaccessinspectorDialogProc@@YGHPAUHWND__@@IIJ@Z@4HA 00412d48     jaccessinspector.obj
 0003:00000d50       _GS_ExceptionRecord        00412d50     MSVCRT:gs_report.obj
 0003:00000da0       _GS_ContextRecord          00412da0     MSVCRT:gs_report.obj
 0003:00001074       ?is_initialized_as_dll@@3_NA 00413074     MSVCRT:utility.obj
 0003:00001075       ?module_local_atexit_table_initialized@@3_NA 00413075     MSVCRT:utility.obj
 0003:00001078       ?module_local_atexit_table@@3U_onexit_table_t@@A 00413078     MSVCRT:utility.obj
 0003:00001084       ?module_local_at_quick_exit_table@@3U_onexit_table_t@@A 00413084     MSVCRT:utility.obj
 0003:00001090       ?g_tss_cv@@3U_RTL_CONDITION_VARIABLE@@A 00413090     MSVCRT:thread_safe_statics.obj
 0003:00001094       ?g_tss_event@@3PAXA        00413094     MSVCRT:thread_safe_statics.obj
 0003:00001098       ?g_tss_mutex@@3U_RTL_CRITICAL_SECTION@@A 00413098     MSVCRT:thread_safe_statics.obj
 0003:000010b0       ?g_sleep_condition_variable_cs@@3P6GHPAU_RTL_CONDITION_VARIABLE@@PAU_RTL_CRITICAL_SECTION@@K@ZA 004130b0     MSVCRT:thread_safe_statics.obj
 0003:000010b4       ?g_wake_all_condition_variable@@3P6GXPAU_RTL_CONDITION_VARIABLE@@@ZA 004130b4     MSVCRT:thread_safe_statics.obj
 0004:000001c0       $R000000                   004141c0     jaccessinspector.exe.res
 0004:00000508       $R000348                   00414508     jaccessinspector.exe.res
 0004:000006a0       $R0004E0                   004146a0     jaccessinspector.exe.res
 0004:000007b0       $R0005F0                   004147b0     jaccessinspector.exe.res
 0004:00001058       $R000E98                   00415058     jaccessinspector.exe.res
